:100000000C946A120C9487120C9487120C94871229
:100010000C9487120C9487120C9487120C94AA1ECD
:100020000C9487120C9487120C9487120C948712EC
:100030000C9415150C9487120C9487120C9487124B
:100040000C9487120C9487120C94071D0C94871241
:100050000C9487120C9487120C9487120C948712BC
:100060000C9487120C9469150C9487120C948712C7
:100070000C9487120C9487120C94E81D0C94871230
:100080000C9487120C9487120C9487123A012A045C
:100090002800290020002100220023002400250040
:1000A0002600270028012802218F28032100280488
:1000B00028052806280728082809280A280B280CBC
:1000C00020802190280D20002100280E20812191E0
:1000D000280F200021922810210028112193281296
:1000E00021002813281428152082281620002817FC
:1000F000281828192194281A2195281B2196281C94
:100100002100281D2083281E2000281F2197282039
:1001100021002821282228232824282528262827AA
:1001200028282829282A2084282B2000282C282D1C
:10013000282E282F283028312832208528332000E7
:10014000283428352836283721982838210028399E
:10015000283A283B283C283D283E283F2840284173
:100160002842284328442845284628472848284923
:10017000284A284B284C284D284E284F28502851D3
:100180002852285328542855285628572858285983
:10019000285A285B285C285D285E285F2860286133
:1001A0002862219928632100286428652866286729
:1001B00028682869286A286B286C286D286E286FA3
:1001C0002870287128722873287428752876287753
:1001D00028782879287A287B287C287D287E287F03
:1001E00028802881288228832884288528862887B3
:1001F00028882889288A288B288C288D288E288F63
:1002000028902891208628922087289320002894DF
:1002100028952896289728982899289A289B289CDA
:10022000289D289E289F219A28A0210028A128A245
:1002300028A328A428A528A628A728A828A928AA4A
:1002400028AB28AC28AD28AE28AF28B028B128B2FA
:1002500028B328B428B528B628B728B828B92088E4
:1002600028BA200028BB208928BC200028BD28BE31
:1002700028BF28C028C128C228C3219B28C4210028
:1002800028C528C628C728C828C928CA28CB28CCEA
:1002900028CD28CE28CF28D028D128D228D328D49A
:1002A00028D528D628D728D828D928DA28DB28DC4A
:1002B00028DD28DE28DF28E028E1208A28E2208BBC
:1002C00028E3200028E428E528E628E728E828E9AC
:1002D00028EA28EB28EC28ED28EE28EF28F028F172
:1002E00028F228F328F428F528F628F728F8208C97
:1002F00028F92000219C28FA219D28FB208D219E91
:1003000028FC208E219F28FD2000210028FE28FFA8
:100310002A012800220123952489250726A42707DE
:10032000280121C72200238026C4270C2802200987
:10033000211C220426AA270A2803200021002200CB
:1003400023A626A02707280428052005238426B4F1
:1003500027092806200022032300248125C026AB7C
:10036000270A280721AE220023952489250726A4E1
:100370002700280821482201238026C4270C2809A9
:1003800020092104220426AA270A280A2000210085
:10039000220023A826A42707280B280C214022206E
:1003A000238026C4270C280D222426C6280E219E31
:1003B000220026C8280F20092102221426AA270A73
:1003C0002810200521002200238426B427092811A3
:1003D000200021012300240125C026AB270A281272
:1003E00021C32395248925072620270028132003CD
:1003F00021C223832626270D281421B3220828157D
:10040000200021C622002395260027082816210057
:1004100023002496250326AA270A2817204221B65E
:100420002380248925072818200021002394260EE4
:100430002819200F238426B42709281A2000239383
:1004400026A82703281B26282700281C2101230073
:10045000240125C026AB270A281D21C52395248900
:10046000250726202700281E210023942600270A7E
:10047000281F260E282020032179220123832626E7
:10048000270D282121322822200021042200238048
:10049000240025FC26AA270A282321002300250062
:1004A000282421A3220D2380249E253B2825204299
:1004B0002157220124892507282620002143220DC7
:1004C00024002538282721082298239524892507E8
:1004D000262427002828204221932201238026AAAF
:1004E000270A28292003217E220423832626270D7C
:1004F000282A200021B02200239526A02707282B98
:1005000021002300240C250426AA270A282C2102D6
:100510002380248625C326AB282D20422197220143
:100520002489250726AA282E200021002200241F26
:100530002504282F21B22395248925072620270466
:1005400028302042218B2204238026AA270A283122
:10055000200021B12200239526A02707283220035E
:100560002175220423832626270D28332005210008
:100570002200238426B42709283420002160230088
:10058000240125C026AB270A283521082298239567
:100590002489250726242700283621BC2200283755
:1005A00021A3220D2300240125C026AB270A2838C9
:1005B0002160220023802400253826AA283921061C
:1005C000229823952489250726242700283A21BE2E
:1005D0002200283B20052100238426B42709283C3B
:1005E000200021602300240125C026AB270A283DD6
:1005F0002142220123952489250726242700283E0D
:10060000210C229826A42707283F21082840216092
:1006100022002300240125C026AB270A2841210CF3
:10062000229823952489250726242700284220057F
:1006300021002200238426B4270928432000238098
:100640002400251026AB270A2844212222012395C5
:10065000248925072624270028452100220023007D
:100660002404251226AA270A2846200321D422057D
:100670002383248925072626270D2847200021606B
:1006800022002300240125C026AB270A284821B3D5
:1006900023952489250726002708284921002300BF
:1006A0002409250026AA270A284A21022380248615
:1006B000253B284B204221DD220524892507284C93
:1006C000200021002200241F2500284D21B323955E
:1006D0002489250726202700284E2100230024975F
:1006E000250326AA270A284F204221E2220523803B
:1006F000248925072850200021102200230024806F
:1007000025CC26AB28512100224023B4248925077B
:1007100026AA27042852220023B02692270928530C
:10072000211422012395260027082854214823A4B8
:10073000262A27002855210022002300240925000D
:1007400026AA270A2856210823802486253B2857D5
:100750002042211122072489250728582000210042
:100760002200241F250028592114220123952489C1
:10077000250726202700285A211626022709285B4C
:100780002100220023002480254826AA270A285C6D
:1007900023A02489250726142709285D24802550B5
:1007A00026A42704285E21162201239524892507E3
:1007B0002700285F210422002300249C257826AAF4
:1007C000270A28602143220D240125C426AB286175
:1007D000210322002415286221002400250026AAD6
:1007E0002863215E2395248925072610270928647C
:1007F00021032300241525C426AB270A28652100E0
:1008000023802400250626AA2866248F25E326AB0C
:100810002867204221CD22072489250726AA286897
:100820002000216022002300240125C026AB286976
:1008300021002380248F250326AA286A204221DD57
:10084000220724892507286B20002143220D23003D
:10085000240125C026AB286C210022002400250499
:1008600026AA286D2003217F2201238324892507BE
:100870002626270D286E2162286F200521002200E0
:10088000238426B4270928702000210623952600FA
:1008900027082871210123002497253B26AA270A2F
:1008A00028722042210E22082380248925072873DC
:1008B0002003213C220B23832626270D28742000A9
:1008C00021032200239526022708287521272300CB
:1008D000248125C426AB270A2876210023802409F9
:1008E000254826AA28772158223423A324892507BE
:1008F000262A270028782100220023A02600270985
:100900002879210723802403253926AA270A287A53
:1009100021042300241C2538287B210723802483DD
:100920002539287C210323952489250726022708B9
:10093000287D21272300248125C426AB270A287E71
:10094000210023802409254826AA287F2158223403
:1009500023A324892507262A270028802106220090
:100960002300248125C0269327012881210023808C
:100970002489254826AA270A2882200221662208DF
:1009800023002400256628832000210022002380E4
:10099000241F2502288421062489250726DC270C0C
:1009A0002885210023AA26AA270A288623B62600FE
:1009B0002708288723802486253B26AA270A2888FB
:1009C00021052489250726DC270C2889210023AA54
:1009D00026AA270A288A23B626002708288B2380E0
:1009E0002486253B26AA270A288C2042217B220820
:1009F00024892507288D20002100220023002401BE
:100A00002582288E2105248125C226AB288F20032C
:100A1000219322082383248925072626270D289041
:100A20002000210522002300248125C02613270150
:100A30002891210023802489254826AA270A289264
:100A40002002217E2208230024002566289320000E
:100A5000210022002380241F2502289421052489B7
:100A6000250726DC270C2895210023AA26AA270A79
:100A7000289623B626002708289723802486253B1E
:100A800026AA270A289821052489250726DC270C71
:100A90002899210023AA26AA270A289A2380241FFE
:100AA0002502289B21012300248125C226AB289CF6
:100AB0002003219322082383248925072626270D36
:100AC000289D200021042200239526122708289E15
:100AD000216023C426AA2704289F210023C02600C2
:100AE000270928A0204221CB2208238026AA270AF2
:100AF00028A12070215422B823952612270828A265
:100B0000200221CC2208238026AA270A28A320031A
:100B100021CA220F23832626270D28A42000210086
:100B200022002300248C250C26AA270A28A52104AC
:100B30002482257828A6210023802489254826128E
:100B4000270428A7200321DE220F2383250726263A
:100B5000270D28A82000210122002300249C2578AD
:100B600026AA270A28A9210023802481254028AA13
:100B7000200321CF220F2383248925072626270D32
:100B800028AB2070210822B8239526A0270428AC82
:100B9000200321D4220F23832626270D28AD2127C9
:100BA000220B28AE2070216322B823952612270835
:100BB00028AF2000210122002380248625CB26ABEC
:100BC000270A28B0204221DD22082489250726AAE9
:100BD00028B1200021182280239526A4270028B2BE
:100BE000200321D9220F23832626270D28B3207026
:100BF000210A22B8239526A0270028B4200221E04C
:100C00002208238026AA270A28B52070210A22B8A4
:100C1000239526A0270028B621542602270828B7A6
:100C200020002118228026A4270028B821002200B5
:100C300023802480254826AA270A28B92070215E0F
:100C400022B82395248925072612270828BA2000D0
:100C50002100220023802409254B26AA270A28BB2D
:100C60002070215F22B823952489250726102708A4
:100C700028BC2000210022002300241C258326AB51
:100C8000270A28BD2003213222092383248925072E
:100C90002626270D28BE20002100220023002482C2
:100CA000258C26AB270A28BF200321252209238370
:100CB000248925072626270D28C0204221BC238011
:100CC00026AA270A28C1200021012200230024018E
:100CD00025C026AB28C22070210F22B82395248975
:100CE00025072620270028C3200321E3220F238382
:100CF0002626270D28C4200521002200238426B49F
:100D0000270928C52000210323952614270828C673
:100D100021A623A4262A270528C7210023A026448C
:100D2000270928C82118226D2380249E257B26AA06
:100D3000270A28C920422113220B2489250728CA03
:100D4000200021AE220023952624270028CB210055
:100D5000220323802487257B26AA270A28CC204229
:100D60002116220B2489250728CD200021AE220040
:100D700023952624270028CE20052100238426B48D
:100D8000270928CF2003210D220B23832626270D98
:100D900028D02000210022002300248026022700E2
:100DA00028D1238024092548261E28D22158223400
:100DB000233324802507262A28D32100220023005C
:100DC0002680271028D421102363262A270028D51F
:100DD0002100236026A8271228D621AF224C230009
:100DE00026C8270C28D7210022002680270528D8CE
:100DF00023802486253B261E270028D92042211C3B
:100E0000220E23002480250728DA200021352229FC
:100E100026C4270C28DB2002211D220E261E2700B7
:100E200028DC2000217F223426C4270C28DD210065
:100E300022002390249F25042610270A28DE230061
:100E4000248425002680271028DF210623632480A0
:100E50002507262A270028E021002380248926AAA6
:100E6000270A28E12005238426B4270928E22070D8
:100E7000216122B823952612270828E320002101AA
:100E800022002380248625C326AB270A28E420429B
:100E900021CE220F2489250726AA28E5207021507B
:100EA00022B823952612270828E6200521002200D3
:100EB000238426B4270928E72070216422B82395CB
:100EC0002612270828E820002101220023802486FA
:100ED00025C326AB270A28E9204221D3220F2489E3
:100EE000250726AA28EA2070215122B82395261228
:100EF000270828EB200521002200238426B4270997
:100F000028EC2070216522B823952612270828EDA9
:100F10002000210122002380248625C326AB270A36
:100F200028EE204221D8220F2489250726AA28EF5F
:100F30002070215222B823952612270828F0200578
:100F400021002200238426B4270928F12070216182
:100F500022B823952602270828F22000210122002A
:100F60002380248625C326AB270A28F3204221DDCF
:100F7000220F2489250726AA28F42070215022B8A0
:100F800023952602270828F5200521002200238426
:100F900026B4270928F6200021012380248625CBAA
:100FA00026AB270A28F7204221E1220F24892507B2
:100FB00026AA28F82000210222002300248125C42B
:100FC00026AB28F9210023802489254826AA28FA5F
:100FD00020052384250726B4270928FB2070214EED
:100FE00022B823952610270828FC20002100220083
:100FF0002380248625C326AB270A28FD204221E72B
:10100000220F2489250726AA28FE200021BB2200C2
:1010100023952620270028FF20052100238426B4BD
:1010200027092A0810013A00643A65BB083A09BB4F
:1010300050105267517705A1180454015523070039
:10104000060C0B03501051005204610F6455655596
:1010500005A11804720113012A2A202020455849AD
:1010600054204D454E555320414E442020202A2ADD
:101070002A2A202052455455524E20544F20504C7D
:101080004159455220202A2A004368616E67652035
:1010900043757272656E74204469726563746F7211
:1010A0007900446973706C6179204E756D62657268
:1010B000206F662046696C65732020696E20437539
:1010C0007272656E74204469726563746F72790020
:1010D00020204368616E676520506C6179657220DD
:1010E0004F75747075742020202020202028766F82
:1010F0006C756D6529206C6576656C0020204368F1
:10110000616E676520506C6179657220426173730E
:10111000202020202020202020202020204C657608
:10112000656C0020204368616E676520506C6179B2
:10113000657220547265626C65202020202020207A
:10114000202020204C6576656C004C6561726E2015
:1011500049522052656D6F746520436F6E74726FD3
:101160006C006A1192115810022D721162118910CF
:101170004F2F7A116A11A2100F2F82117211D01005
:10118000032D8A117A11FC106D2D921182112311F9
:10119000CD2D62118A114A112A332020202020509F
:1011A0006F77657220286F6E2F6F6666290020208A
:1011B0002020202020202020506C61790020202039
:1011C0002020202020202053746F70002020202019
:1011D0002020202020204E65787400202020202010
:1011E00020202020204261636B002020204D6F646E
:1011F00065202872616E646F6D2C20657463290010
:10120000081228129A11350110120012AE11B50100
:1012100018120812BD11350220121012CC1135031C
:1012200028121812DB11B50300122012EA11B502C0
:101230000D0A0A53746172742E203F20666F72206B
:1012400068656C702E0D0A000A0D0A0A4552524F4D
:10125000523A2024000A0D0052616E646F6D200026
:101260004F6666004F6E0052657065617420004FD6
:101270006666004F6E005C48304120202020202010
:101280002020202020005C483142202020202020E7
:101290002020202020005C483243202020202020D5
:1012A0002020202020005C483344202020202020C3
:1012B0002020202020005C483445202020202020B1
:1012C0002020202020005C4835462020202020209F
:1012D0002020202020005C4836472020202020208D
:1012E0002020202020005C4837482020202020207B
:1012F0002020202020005C48384920202020202069
:101300002020202020005C48394A20202020202056
:101310002020202020005C483A4B20202020202044
:101320002020202020005C483B4C20202020202032
:101330002020202020005C48402020202020202049
:101340002020202020005C48412020202020202038
:101350002020202020005C48422020202020202027
:101360002020202020005C48432020202020202016
:101370002020202020005C48442020202020202005
:101380002020202020005C484520202020202020F4
:101390002020202020005C4846672020202020209C
:1013A0002020202020005C484720202020202020D2
:1013B0002020202020005C484820202020202020C1
:1013C0002020202020005C484920202020202020B0
:1013D0002020202020005C484A202020202020209F
:1013E0002020202020005C484B202020202020208E
:1013F0002020202020005C48502020202020202079
:101400002020202020005C48512020202020202067
:101410002020202020005C48522020202020202056
:101420002020202020005C48532020202020202045
:101430002020202020005C48542020202020202034
:101440002020202020005C48552020202020202023
:101450002020202020005C48562020202020202012
:101460002020202020005C48572020202020202001
:101470002020202020005C485820202020202020F0
:101480002020202020005C485920202020202020DF
:101490002020202020005C485A20202020202020CE
:1014A0002020202020005C485B20202020202020BD
:1014B00020202020200052656164792020202020F7
:1014C000202020202020202020202020202020201C
:1014D000202020202020202020202020202020200C
:1014E0002020004F6E65206D6F6D656E7420706CEE
:1014F000656173652E2E2E002020204672616E6B72
:101500002773204D503320506C6179657200436F12
:10151000756E74696E67204D50332046696C657333
:1015200020202020202000204D50332066696C654B
:101530007320666F756E642E004275696C64696E07
:1015400067204661737446696E64207461626C65DD
:1015500020000D0A436F6D6D656E63696E672041F3
:10156000565220506F727473204269747320546510
:101570007374732E0D0A004552524F52202D207065
:10158000696E2074696564206C6F772E2000455267
:10159000524F52202D204170706172656E74207020
:1015A000696E2073686F72742E20506F72742041C0
:1015B000206F75747075742076616C756520776125
:1015C00073203078002E20556E65787065637465E1
:1015D000642070696E206C6F7720666F756E642072
:1015E0006F6E20004552524F52202D204170706185
:1015F00072656E742070696E2073686F72742E202D
:10160000506F72742042206F75747075742076610B
:101610006C756520776173203078002E20556E65DB
:10162000787065637465642070696E206C6F7720D4
:10163000666F756E64206F6E20004552524F5220C7
:101640002D204170706172656E742070696E207318
:10165000686F72742E20506F72742043206F7574FF
:101660007075742076616C756520776173203078B1
:10167000002E20556E65787065637465642070690E
:101680006E206C6F7720666F756E64206F6E200021
:101690004552524F52202D204170706172656E7418
:1016A0002070696E2073686F72742E20506F727490
:1016B0002044206F75747075742076616C75652098
:1016C000776173203078002E20556E6578706563E1
:1016D0007465642070696E206C6F7720666F756E1C
:1016E00064206F6E20004552524F52202D204170D1
:1016F000706172656E742070696E2073686F7274A9
:101700002E20506F72742045206F75747075742090
:1017100076616C756520776173203078002E2055D6
:101720006E65787065637465642070696E206C6F97
:101730007720666F756E64206F6E20004552524FA1
:1017400052202D204170706172656E742070696E38
:101750002073686F72742E20506F72742046206F51
:1017600075747075742076616C756520776173206F
:101770003078002E20556E6578706563746564203E
:1017800070696E206C6F7720666F756E64206F6E67
:1017900020004552524F52202D20417070617265D9
:1017A0006E742070696E2073686F72742E20506F93
:1017B00072742047206F75747075742076616C7533
:1017C0006520776173203078002E20556E65787023
:1017D00065637465642070696E206C6F7720666F36
:1017E000756E64206F6E20004552524F52202D209E
:1017F00070696E207469656420686967682E2000CE
:1018000041565220506F7274732042697473205491
:101810006573747320436F6D706C657465642E0D11
:101820000A00506F7274200020426974206E756D3A
:1018300062657220000D0A00436F6D6D656E63690D
:101840006E6720486172646469736B2054657374B9
:10185000732E0D0A0057616974696E6720666F7296
:10186000206472697665206E6F7420627573792EBC
:1018700020004472697665207374617475732072F8
:10188000656769737465723A203078000D0A4F4BB2
:101890002C206472697665206E6F206C6F6E6765B0
:1018A0007220627573792E0D0A004552524F523ADA
:1018B0002053746174757320616E6420416C74658B
:1018C000726E6174652053746174757320726567FC
:1018D000697374657273206E6F7420746865207309
:1018E000616D652E0D0A0053746174757320726505
:1018F0006769737465723A20307800202020416C4B
:101900007465726E617465205374617475732072AE
:10191000656769737465723A203078000D0A41205A
:101920007479706963616C2053746174757320728B
:10193000656769737465722076616C75652069737B
:1019400020307835302E0D0A004552524F52206318
:101950006F6E6669726D696E6720736563746F720E
:1019600020636F756E742072656769737465722C7D
:10197000206164647265737320307835372E0D0AE8
:101980000044617461207772697474656E207761B8
:101990007320307841412E2044617461207265616A
:1019A0006420776173203078002E0D0A0048617240
:1019B000646469736B20546573747320436F6D7036
:1019C0006C657465642E0D0A0057726974696E67E0
:1019D0002030784141277320746F2074686520534C
:1019E0006563746F7220436F756E7420526567690A
:1019F0007374657220666F72657665722E0D0A00CB
:101A000052656164696E67207468652053746174FF
:101A1000757320526567697374657220666F7265AD
:101A20007665722E0D0A0049522064656275672042
:101A3000666C6167207365742E2028506F7765721D
:101A40002D6F666620746F20636C6561722E290DA0
:101A50000A000D0A556E6B6E6F776E20636F6D6DA9
:101A6000616E642E000D0A446562756720506F72C6
:101A70007420436F6D6D616E6473206172653A0A04
:101A80000D0A003F20202D207072696E742074684A
:101A900065736520636F6D6D616E64730D0A00651B
:101AA00020202D2064756D7020636F6E74656E74D8
:101AB00073206F6620656570726F6D0D0A0064207B
:101AC000202D2064756D7020736F6D6520646973BF
:101AD0006B647269766520646562756720696E66FD
:101AE0006F726D6174696F6E0D0A006820202D2081
:101AF00064756D7020736F6D652064656275672015
:101B0000696E666F2028737461636B2064756D70F5
:101B100029207468656E2068616E67202870726F76
:101B2000636573736F722073746F70706564290DD1
:101B30000A006920202D20656E61626C6520647545
:101B40006D70696E67206F662049522072656D6FF7
:101B500074652D636F6E74726F6C20706572696F3F
:101B6000642076616C75657320647572696E672098
:101B7000747261696E696E670D0A007020202D20F5
:101B8000746573742049444520506F7274732062E9
:101B900069747320776865726520706F737369620A
:101BA0006C652E20484152444449534B204D5553B7
:101BB0005420424520554E504C55474745442E0D24
:101BC0000A007420202D20746573742074686520C9
:101BD000686172646469736B20696E7465726661B2
:101BE00063652E20486172646469736B206D757340
:101BF0007420626520706C756767656420696E2E5D
:101C00000D0A007720202D20506572666F726D20BE
:101C1000726570656174656420777269746573209C
:101C2000746F2074686520686172646469736B2ED8
:101C30000D0A007220202D20506572666F726D2093
:101C40007265706561746564207265616473206695
:101C5000726F6D2074686520686172646469736B6B
:101C60002E0D0A000D0A000A0D537461636B20509B
:101C70006F696E7465722076616C75653A20240018
:101C80000A0D00537461636B2064756D703A2024F3
:101C900020000A0D000A0D00506C61796572206801
:101CA000616C7465642E0D0A00202020205553427B
:101CB00020506F727420496E205573650020506C5F
:101CC00061796572207265737461727473206166E4
:101CD000746572202020555342206361626C652038
:101CE000756E706C75676765642E000D0A0A0A557B
:101CF000534220706F727420696E207573652E0DCB
:101D00000A00506C61796572207265737461727437
:101D100073207768656E2055534220756E706C7520
:101D2000676765642E0D0A0A0055534220706F7272
:101D30007420756E706C75676765642E20526573CC
:101D400074617274696E6720706C617965722E0DB2
:101D50000A0A00537461636B20506F696E74657278
:101D60002076616C75653A2024000A0D0053746179
:101D7000636B2064756D703A202420000A0D000DFD
:101D80000A4449534B44524956452044454255471D
:101D900020494E464F524D4154494F4E0D0A004680
:101DA000696E6466696C652063757272656E742015
:101DB0006469726563746F727920636C757374659E
:101DC000723A2024000D0A0046696E6466696C65EB
:101DD0002063757272656E74206F66667365742019
:101DE000696E746F207468697320636C75737465B1
:101DF000723A2024000D0A0053747265616D6669A1
:101E00006C652053746174653A2024000D0A004308
:101E1000616C634E657874436C757374657220539E
:101E2000746174653A2024000D0A0043616C634EAE
:101E3000657874436C757374657220736563746F31
:101E4000722069742773207365656B696E672074EF
:101E50006F3A2024000D0A005365656B5365637467
:101E60006F722053746174653A2024000D0A004497
:101E70007269766520737461747573207265676921
:101E8000737465723A2024000D0A00447269766505
:101E9000206572726F722072656769737465723A39
:101EA0002024000D0A00536563746F7273207065FF
:101EB0007220636C75737465723A2024000D0A00F9
:101EC00046415420737461727420736563746F7239
:101ED0003A2024000D0A0044495220737461727440
:101EE00020736563746F723A2024000D0A00466502
:101EF00065645354636F6465635F436F6D6D616EBA
:101F0000643A2024000D0A0046696C65204E756D08
:101F10006265723A2024000D0A000D0A44756D7046
:101F2000206F662074686520647269766527732067
:101F3000426F6F7420506172616D657465722042EA
:101F40006C6F636B3A0D0A002000200020000D0A20
:101F5000000D0A000D0A46697273742033322D6237
:101F6000797465207265636F726420696E20637591
:101F70007272656E74206469726563746F72793A07
:101F80000D0A00200020000D0A000D0A002020206C
:101F90002020202020202020202020202020202041
:101FA0002020202020000D0A454550524F4D20434F
:101FB0006F6E74656E747320696E204865783A0D93
:101FC0000A00202000200020000D0A000D0A004514
:101FD00052524F52202D2043616E6E6F7420506C10
:101FE00061792E202020204E6F204D5033206669CD
:101FF0006C657320696E2063757272656E742064FF
:1020000069726563746F72792E004E6F7720706C01
:102010006179696E673A202020202020202020202E
:1020200020202020202020202020202020202020B0
:102030002020202020202020200046696E64466950
:102040006C65206572726F7220696E20506C6179C8
:1020500046696C65416E64446973706C61792E20C9
:1020600046696C65206E756D6265723A2024000DBC
:102070000A00536F6E672053746570203D20002066
:10208000202020204D656E752046756E6374696F43
:102090006E7320202020202020205570202F2044E7
:1020A0006F776E202F2053656C656374202020208D
:1020B0002020202020200020204368616E676520BA
:1020C0004F7574707574204C6576656C20202020E7
:1020D00020205570202F20446F776E202F205365CD
:1020E0006C65637420202044656661756C7420699A
:1020F000732032353520286D6178696D756D292022
:10210000002020204368616E676520426173732060
:102110004C6576656C202020202020205570202FD3
:1021200020446F776E202F2053656C6563742020E8
:102130002020202020202044656661756C74206971
:1021400073203020202020202000202020436861A0
:102150006E676520547265626C65204C6576656CAF
:1021600020202020205570202F20446F776E202FB4
:102170002053656C656374202020202020202020BF
:1021800044656661756C74206973203020202020BE
:102190002020002D3138206442002D31362E35208C
:1021A0006442002D3135206442002D31332E35201C
:1021B0006442002D3132206442002D31302E352012
:1021C0006442002D39206442002D372E35206442B0
:1021D000002D36206442002D342E35206442002D1F
:1021E00033206442002D312E3520644200302064BB
:1021F00042002B312E35206442002B3320644200F4
:102200002B342E35206442002B36206442002B37BD
:102210002E35206442002B39206442002B31302EB1
:1022200035206442002B3132206442002B31332EA2
:1022300035206442002B3135206442002B31362E8C
:1022400035206442002B313820644200696E76618B
:102250006C69642076616C7565004E756D6265729F
:10226000206F66204D50332066696C657320696E5F
:10227000202063757272656E742064697265637480
:102280006F72790069733A2000507265737320533E
:10229000454C45435420746F20657869742E0020A6
:1022A0002020204368616E6765204469726563740D
:1022B0006F7279202020202020205570202F20446C
:1022C0006F776E202F2053656C65637400204E6F0E
:1022D000204469726563746F7269657320466F7517
:1022E0006E642E20202050726573732053454C4538
:1022F000435420746F20657869742E002E2E2020A0
:1023000020202020005570204F6E652044697265A2
:1023100063746F7279204C6576656C002E202020E6
:10232000202020200053656C6563742074686973F5
:10233000204469726563746F7279002E202020201A
:102340002020202E20202000526F6F7420446972BC
:102350006563746F72790043686F6F73652066758B
:102360006E6374696F6E20746F20747261696E2081
:1023700020205570202F20446F776E202F2053652A
:102380006C6563742000486F6C642072656D6F74B7
:102390006520636F6E74726F6C20202020203330B4
:1023A00020636D2066726F6D204D503320706C611C
:1023B00079657220202049522072656369657665CF
:1023C00072207468656E2070726573732020726568
:1023D0006D6F746520636F6E74726F6C20627574BC
:1023E000746F6E2E00495220636F646520726563BE
:1023F00065697665642E00446F20796F7520776972
:10240000736820746F20747261696E2020202061CF
:102410006E6F746865722066756E6374696F6E3F67
:102420000053656C6563743D7965732C20206F746F
:10243000686572733D6E6F000D0A5374617274208B
:102440006F6620495220706572696F6420726177EF
:1024500020646174610D0A004E756D626572206FB3
:10246000662072617720706572696F64733A20002C
:102470000D0A56616C7565206F66205420286269CC
:102480007420706572696F64293A20000D0A4E75D8
:102490006D626572206F6620706572696F6473206B
:1024A000696E2049522073657175656E63653A20C7
:1024B000000D0A000D0A00456E64206F6620495227
:1024C00020706572696F6420726177206461746145
:1024D0000D0A000011241FBECFEFD0E1DEBFCDBF3B
:1024E00011E0A0E0B1E0ECECF8E700E00BBF02C0C7
:1024F00007900D92A030B107D9F710E1A0E0B1E04C
:1025000001C01D92A830B107E1F70C9489120C9418
:102510000000CFEFD0E1DEBFCDBF0E94D3130E94F9
:1025200040350E94DA150E94E0150E94753610921F
:1025300019010E94261578940E94C8360E94FB1447
:102540000E9442350E94E8130E94C9150E94B815E6
:102550008AEF0E94B6360E94A4380E94C8380E94B2
:1025600094140E94911380E392E10E94F41C88E08D
:1025700090E00E94353C9927AA27BB27182F0027F7
:10258000FF24EE2487E090E00E94353C9927AA279B
:10259000BB27DC0199278827E80EF91E0A1F1B1F9D
:1025A00086E090E00E94353C9927AA27BB27BA2FE6
:1025B000A92F982F8827E80EF91E0A1F1B1F85E0F8
:1025C00090E00E94353CE80EF11C011D111DE092C7
:1025D000540FF092550F0093560F1093570F8091A0
:1025E000540F9091550FA091560FB091570F00972F
:1025F000A105B10571F08091540F9091550FA091F4
:10260000560FB091570F8F5F9F4FAF4FBF4F09F0DD
:102610004FC082E090E0A0E0B0E08093540F909330
:10262000550FA093560FB093570F8091540F909170
:10263000550FA091560FB091570F682F85E090E08D
:102640000E9445268091540F9091550FA091560FEE
:10265000B091570F892F9A2FAB2FBB27682F86E099
:1026600090E00E9445268091540F9091550FA091C3
:10267000560FB091570FCD01AA27BB27682F87E0CF
:1026800090E00E9445268091540F9091550FA091A3
:10269000560FB091570F8B2F9927AA27BB27682F6A
:1026A00088E090E00E9445260E94F6150E94CF1611
:1026B0000E9473190E94A7150E94B3370E945439D3
:1026C0000E94751F0E94CC230E94751F0E945439DE
:1026D0000E9480230E94751F0E94321E0E9454395E
:1026E0000E94751FEBCF1F93182F8CE50E948E362A
:1026F00080E40E948E3680E20E948E3680E30E9443
:102700008E3688E492E10E94F41C812F0E94973655
:1027100085E592E10E94F41C0E94DD1F0E94D137E2
:10272000FFCF84E080930101109217018FEF809317
:1027300012010E94A8131092140181E090E090937E
:10274000160180931501909303018093020108956F
:1027500061E088E00E94072261E088E00E94242274
:1027600088E592E10E94151E80911701882319F4D3
:1027700080E692E102C084E692E10E94151E6FE0BD
:1027800088E00E94242287E692E10E94151E809133
:102790001201882319F48FE692E102C083E792E1E7
:1027A0000E94151E089582B18B6F82B982B18F711C
:1027B00082B98CE30E94B6361A98129A8CE30E9472
:1027C000B6368AB780638ABF89B7806489BF0895A7
:1027D0008CE50E948E3680E40E948E3680E20E9454
:1027E0008E3680E30E948E368CE50E948E3681E420
:1027F0000E948E3681E30E948E368CE50E948E36D2
:102800008BE50E948E3686E792E10E94151E86E8CF
:1028100092E10E94151E86E992E10E94151E86EA49
:1028200092E10E94151E86EB92E10E94151E86EC35
:1028300092E10E94151E86ED92E10E94151E86EE21
:1028400092E10E94151E86EF92E10E94151E86E01D
:1028500093E10E94151E86E193E10E94151E86E217
:1028600093E10E94151E86E393E10E94151E86E403
:1028700093E10E94151E86E593E10E94151E86E6EF
:1028800093E10E94151E86E793E10E94151E86E8DB
:1028900093E10E94151E86E993E10E94151E86EAC7
:1028A00093E10E94151E86EB93E10E94151E86ECB3
:1028B00093E10E94151E86ED93E10E94151E86EE9F
:1028C00093E10E94151E86EF93E10E94151E86E09B
:1028D00094E10E94151E86E194E10E94151E86E295
:1028E00094E10E94151E86E394E10E94151E86E481
:1028F00094E10E94151E86E594E10E94151E86E66D
:1029000094E10E94151E86E794E10E94151E86E858
:1029100094E10E94151E86E994E10E94151E86EA44
:1029200094E10E94151E08950F931F93CF93DF9398
:10293000B89AC09A139A82B18F7182B91B981B986A
:102940001B981B981B981B981B981B981B9ACFE2EF
:10295000D5E781B12197D7FFFCCF88EF8093710035
:1029600088E28093700010920001C0E0D0E0FE0188
:10297000E457FF4F21961491FE01E457FF4F219633
:102980008491682F812F0E94221F082F103111F48B
:102990000E94DF1C002319F0802F0E94731390E027
:1029A00081B19F5F9837E0F38FE0CC3CD807FCF211
:1029B00087B3866087BB89E58DB91FB80E94DF1C8D
:1029C00068EB87E70E94221F0E94DF1C6BE088E70C
:1029D0000E94221F0E94DF1C6AEF89E70E94221FCB
:1029E0000E94DF1C60E08AE70E94221FDF91CF91E6
:1029F0001F910F91089581E083BF109213011FBCB6
:102A00008BE08EBD81E68BBD88EA8ABD87B7806189
:102A100087BF179810928B0084E880938A0080917A
:102A20007D00806280937D0008951F920F920FB603
:102A30000F9211248F93809113018F5F8093130164
:102A40008F910F900FBE0F901F9018951F93CF93EB
:102A5000DF93C5E3D1E015E0CE010E94353C8F3F06
:102A600021F460E0CE010E944526C058DF4F11508E
:102A700098F710921B0110921A0115E0E12FFF2721
:102A8000E45FFE4F10821150C8F761E486E391E0E5
:102A90000E94452664E486EB91E00E94452663E4AB
:102AA00086E392E00E94452667E686E393E00E9473
:102AB000452666E486EB93E00E94452662E486EBB9
:102AC00092E00E94452610921801DF91CF911F914C
:102AD00008951F920F920FB60F9211242F933F93D8
:102AE0004F935F936F937F938F939F93AF93BF9316
:102AF000EF93FF93109289001092880080918A00D2
:102B000090E4892780938A0080E280937C00209162
:102B10008000809181009927982F8827820F911D2E
:102B200090931B0180931A010E94DD22FF91EF9187
:102B3000BF91AF919F918F917F916F915F914F91D5
:102B40003F912F910F900FBE0F901F9018958CE51D
:102B50000E948E3682E40E948E3680E20E948E367B
:102B600082E20E948E3686EB94E10E94151E089543
:102B70008CE50E948E3682E40E948E3680E20E94AE
:102B80008E3683E20E948E3683EE94E10E94151EFB
:102B900008958CE50E948E3682E40E948E3680E293
:102BA0000E948E3680E20E948E3688EF94E10E9469
:102BB000151E0895BC9AC4980895C49ABC9A0895A5
:102BC00080916200806280936200809161008062E7
:102BD000809361000895809162008F7D80936200F0
:102BE0008091610080628093610008950F931F932C
:102BF00061E082E00E9424228EE095E10E94151E91
:102C00000E941E168C01682F83E090E00E944526EA
:102C1000812F9927682F84E090E00E94452661E08B
:102C200082E00E94242261E0C8010E94392287E2EA
:102C300095E10E94151E1F910F910895BF92CF92AA
:102C4000DF92EF92FF920F931F93CF931092800F1A
:102C50000E9454398091680F882331F00E945439C2
:102C60008091680F8823D1F780E391E00E94653559
:102C70008FEF9FEFAFEFBFE08093041090930510AC
:102C8000A0930610B09307108091540F9091550FA8
:102C9000A091560FB091570F8093640F9093650FDA
:102CA000A093660FB093670F80E391E090936D0F50
:102CB00080936C0F81E08093800F0E9454390E94B2
:102CC0005439CC24DD240DC00E9454398091680F02
:102CD000882339F480E391E00E943136809708F42C
:102CE00054C080E391E00E943136809768F380E31E
:102CF00091E00E947435182F882371F48093800F1F
:102D00008091680F882309F440C00E945439809153
:102D1000680F8823D1F739C0C7E080E391E00E94B3
:102D20007435C150D1F780E391E00E947435B82E1C
:102D300080E391E00E947435E82E80E391E00E94E8
:102D40007435F82E80E391E00E947435082FC4E1B9
:102D500080E391E00E947435C150D1F7153E91F0A7
:102D60008DE4B81679F480E5E81661F483E3F8168B
:102D700049F4802F99278E719070892B19F408944B
:102D8000C11CD11C0E945439ACCFC601CF911F91F8
:102D90000F91FF90EF90DF90CF90BF9008952F920A
:102DA0003F924F925F926F927F928F929F92AF92DB
:102DB000BF92CF92DF92EF92FF920F931F93CF9328
:102DC000DF93CDB7DEB727970FB6F894DEBF0FBEFF
:102DD000CDBF61E083E00E94242289E395E10E9457
:102DE000151E29E030E02E833F83E090540FF090D1
:102DF000550F0091560F1091570F8824992441E0E8
:102E000050E04C835D8314018A829B8284E090E0D1
:102E10000E94353C9927B82EAA2483E090E00E94B6
:102E2000353CA80EB11C55E6A516B10408F04EC0FD
:102E3000DD248E819F81FC013196EE83FF8361E06A
:102E40000E9445268E819F819C012F5F3F4F2E83DC
:102E50003F8360E00E9445268E819F81AC014F5FD9
:102E60005F4F4E835F836E2D0E944526BB27A12FA7
:102E7000902F8F2D2E813F81F9013196EE83FF83B4
:102E8000682FC9010E944526C801AA27BB272E81A9
:102E90003F81A9014F5F5F4F4E835F83682FC90158
:102EA0000E944526812F9927AA27BB272E813F8183
:102EB000F9013196EE83FF83682FC9010E944526F0
:102EC000D394F1E3FD1508F0B4CF6FC10894A108C5
:102ED000B108C50162E370E00E94523C5B011092B0
:102EE00000011092800F0E9454398091680F88234E
:102EF00031F00E9454398091680F8823D1F780E324
:102F000091E00E9465358FEF9FEFAFEFBFE08093B8
:102F1000041090930510A0930610B0930710E09250
:102F2000640FF092650F0093660F1093670F80E3B4
:102F300091E090936D0F80936C0F82E08093800FEF
:102F40000E9454390E9454390E94543922E3298343
:102F50008114910409F062C00DC00E94543980911F
:102F6000680F882339F480E391E00E94313604979A
:102F700008F41BC180E391E00E943136049768F3A6
:102F800080E391E00E947435E82EFF24002711278A
:102F900080E391E00E9474359927AA27BB27BA2FB6
:102FA000A92F982F8827E80EF91E0A1F1B1F80E300
:102FB00091E00E9474359927AA27BB27DC01992745
:102FC0008827E80EF91E0A1F1B1F80E391E00E946C
:102FD00074359927AA27BB27B82FAA2799278827AE
:102FE000E80EF91E0A1F1B1F8091FA0F882E9924E4
:102FF000982C8824990C2A803B800894211C311C31
:103000000DC00E9454398091680F882339F480E301
:1030100091E00E943136809708F4C7C080E391E0C8
:103020000E943136809768F380E391E00E94743506
:10303000C82E882371F48093800F8091680F8823B5
:1030400009F4B3C00E9454398091680F8823D1F7E6
:10305000ACC037E0D32E80E391E00E947435DA945F
:10306000D1F780E391E00E947435482E80E391E02F
:103070000E947435582E80E391E00E947435682ECA
:1030800080E391E00E947435782E24E1D22E80E313
:1030900091E00E947435DA94D1F735EEC316A1F0B1
:1030A0004DE4441689F450E5551671F483E368162F
:1030B00059F4872D99278E719070892B29F4EA8114
:1030C000FB813196EA83FB8320EE3FEF820E931E55
:1030D0000E9454394A815B818C819D814817590730
:1030E00009F053C08E819F81FC013196EE83FF83EE
:1030F000622D0E944526832D99272E813F81A901AB
:103100004F5F5F4F4E835F83682FC9010E94452642
:103110008E819F81FC013196EE83FF836E2D0E948C
:103120004526BB27A12F902F8F2D2E813F81A901EE
:103130004F5F5F4F4E835F83682FC9010E94452612
:10314000C801AA27BB272E813F81F9013196EE8362
:10315000FF83682FC9010E944526812F9927AA273E
:10316000BB272E813F81A9014F5F5F4F4E835F8355
:10317000682FC9010E9445268C819D818A0D9B1D67
:103180008C839D83998191509983E981EE2309F085
:10319000DFCEE093800F8091680F882331F00E948A
:1031A00054398091680F8823D1F727960FB6F89489
:1031B000DEBF0FBECDBFDF91CF911F910F91FF906A
:1031C000EF90DF90CF90BF90AF909F908F907F90C7
:1031D0006F905F904F903F902F900895CF93DF9323
:1031E00084E090E00E94353C9927D82FCC2783E0DB
:1031F00090E00E94353CC80FD11DCE010E9452269E
:103200009093160180931501CA30D10530F481E006
:1032100090E09093030180930201CC33D10538F400
:1032200087E090E0909303018093020134C02EE187
:1032300030E0CE01B9010E94523C709303016093CB
:10324000020180910201909103014E9720F4309386
:103250000301209302018091020190910301880FE4
:10326000991F0E9452269C018091020190910301B6
:10327000820F931F909303018093020180910201BA
:10328000909103018C179D0730F02197D093030193
:10329000C093020121968091020190910301019750
:1032A000F9F02091020130910301CE01B9010E9491
:1032B000523CBC01892B29F0CE010E94523C892B43
:1032C00079F4809102019091030101979093030199
:1032D000809302018091020190910301019709F707
:1032E000DF91CF910895CF9380E090E00E94353C2C
:1032F000C82F8F3F81F4C0E06C2F80E090E00E94E7
:1033000045266C2F81E090E00E9445266C2F82E0DC
:1033100090E00E94452681E00E94B6366C2F86E43C
:103320000E94221F882319F0845C0E94731381E09D
:103330000E94B6366C2F88E40E94221F882319F061
:103340008A5B0E94731381E090E00E94353CC82F95
:103350008D50873E30F4C0E06C2F81E090E00E94F9
:10336000452681E00E94B6366C2F8CE70E94221F12
:10337000882319F0805B0E94731382E090E00E9422
:10338000353CC82F8D50873E30F4C0E06C2F82E072
:1033900090E00E94452681E00E94B6366C2F8BE7B4
:1033A0000E94221F882319F0865A0E94731381E01D
:1033B0000E94B6360E94EB2ECF910895CF92EF92E5
:1033C0000F931F93CF9382E595E10E94F41C8AB37B
:1033D0001ABA8BB39FEF9BBB87B38F7087BB88B341
:1033E000806F88BB84B314BA85B395BB81B38F70EB
:1033F00081BB82B3806F82BB14981C9A809161005C
:10340000807280936100809162008F6D8093620072
:1034100080916400807E80936400809165008F615C
:10342000809365006FE1C62E5FEDE52E00E120EF91
:10343000492F622F892F0E94F91B082F882309F436
:103440004EC087E795E145C08EE895E10E94F41CE7
:103450008C2F0E94973685EC95E13BC084EE95E178
:103460000E94F41C8C2F0E9497368BE196E131C0AC
:103470008AE396E10E94F41C8C2F0E94973681E724
:1034800096E127C080E996E10E94F41C8C2F0E94EF
:10349000973687EC96E11DC086EE96E10E94F41CFB
:1034A0008C2F0E9497368DE197E113C08CE397E152
:1034B0000E94F41C8C2F0E94973683E797E109C085
:1034C00082E997E10E94F41C8C2F0E94973689ECC8
:1034D00097E10E94F41C802F0E94DE1B69C111E05D
:1034E0001ABBC12FC095CBBB4FE1C42E3FEDE32EDD
:1034F00000E120EF4FEF622F8C2F0E94F91B082F65
:10350000882309F0A1CF110F59F78AB30ABB8BB3F7
:103510008FEF8BBB10E187B38F7087BB87B3812B95
:1035200087BB88B3806F88BBC12FC09588B38C23BD
:1035300088BB8C2F807F2FE1C22E9FEDE92E00E10A
:1035400020EF4FEF682F842F0E94F91B082F88234C
:1035500009F084CF110FF9F687B38F7087BB88B35A
:10356000806F88BB11E014BBC12FC095C5BB0FE1B4
:10357000C02EBFEDEB2E00E120EF4C2F622F8FEF1E
:103580000E94F91B082F882309F072CF110F59F7F9
:1035900084B304BB85B38FEF85BB10E181B38F701B
:1035A00081BB81B3812B81BB82B3806F82BBC12F72
:1035B000C09582B38C2382BB8C2F807FAFE1CA2E53
:1035C000FFEDEF2E00E1282F4FEF60EF842F0E94D8
:1035D000F91B082F882309F055CF110FF9F681B395
:1035E0008F7081BB82B3806F82BB10E1149882B16F
:1035F000812B82B91C9AC12FC09583B18C2383B9CA
:103600008C2F8071EFE1CE2E7FEDE72E082F20EF7B
:103610004FEF622F842F0E94F91B082F882309F097
:103620003BCF110F103111F314981C9A11E0109335
:103630006100C12FC095C09362008C2F8F7D6FE118
:10364000C62EE82E00E120EF4FEF622F842F0E945C
:10365000F91B082F882309F029CF110F41F780911A
:103660006100807280936100809162008F6D809311
:10367000620010E180916400807E809364008091FC
:103680006400812B80936400809165008F6180933A
:103690006500C12FC095809165008C2380936500E3
:1036A0008C2F8F71C82E5FEDE52E00E120EF4FEFDC
:1036B000622F842F0E94F91B082F882309F000CF66
:1036C0001695C1F680916400807E8093640080919D
:1036D00065008F61809365008BB30BBB88B38F70DF
:1036E00088BB85B305BB82B38F7082BB1C98809169
:1036F000620080728093620080916500807E80937A
:1037000065008AB3CFEFCABB87B3806F87BB84B332
:10371000C4BB81B3806F81BB149A809161008E29F4
:1037200080936100809164008F61809364004FE119
:10373000C42E00E120EF4C2F622F8C2F0E94311CF1
:10374000082F882339F088EE97E10E94F41C802F1F
:103750000E94DE1B8AB31ABB87B38F7087BB84B30A
:1037600014BB81B38F7081BB14988091610080720B
:103770008093610080916400807E809364008BB3AD
:10378000CBBB88B3806F88BB85B3C5BB82B3806F6A
:1037900082BB1C9A809162008F6D80936200809141
:1037A00065008F618093650080E098E10E94F41CC1
:1037B000CF911F910F91EF90CF9008951F93182FE5
:1037C00082E298E10E94F41C812F82958F70805CC8
:1037D0000E94823688E298E10E94F41C1F70105DFE
:1037E000812F0E94823685E398E10E94F41C1F918C
:1037F0000895CF92EF920F9390E139B3309538232B
:1038000011F590E236B330953623E9F490E333B303
:1038100030953423C1F490E430B33095322399F4D9
:1038200090E531B13095302371F490E630B13095A8
:103830003E2149F490E73091630030953C2119F422
:1038400080E090E00AC080E030FD04C036958F5FD4
:1038500030FFFCCF982B892F99270F91EF90CF90B5
:103860000895CF92EF920F9390E139B33823E1F4AA
:1038700090E236B33623C1F490E333B33423A1F49A
:1038800090E430B3322381F490E531B1302361F418
:1038900090E630B13E2141F490E7309163003C2145
:1038A00019F480E090E00AC080E030FD04C0369555
:1038B0008F5F30FFFCCF982B892F99270F91EF90C6
:1038C000CF9008951F93CF9388E398E10E94F41C52
:1038D00085E598E10E94F41C82E798E10E94F41CBF
:1038E0008FE70E9414370E9497368FE70E941437A3
:1038F00087FDFBCF8CE898E10E94F41C8FE70E94C3
:103900001437C82F87EB0E941437182FC817B1F04F
:103910008AEA98E10E94F41C87EE98E10E94F41C68
:103920008C2F0E9497368BEF98E10E94F41C812F18
:103930000E9497368CE199E10E94F41C6AEA87E5BF
:103940000E943D3765E58FE50E943D376FE087E6D1
:103950000E943D3760EF8FE60E943D376CEE87E7AF
:103960000E943D3787E50E941437C82F8A3A79F0C4
:1039700089E499E10E94F41C81E899E10E94F41C19
:103980008C2F0E94973689EA99E10E94F41C8DEAF7
:1039900099E10E94F41CCF911F91089589EC99E15F
:1039A0000E94F41C6AEA87E50E943D37FBCF80E065
:1039B0009AE10E94F41C8FE70E941437FCCF90E03C
:1039C00081B19F5F9F3FE1F70895CF93DF93EC01B3
:1039D0008881882331F089910E94823688818823EA
:1039E000D1F7DF91CF910895CF93DF93EC01FC01E4
:1039F0008491882349F0FE0184910E9482362196A9
:103A0000FE0184918823B9F7DF91CF9108951F9229
:103A10000F920FB60F9211242F933F934F935F9302
:103A20006F937F938F939F93AF93BF93EF93FF9386
:103A30008CB199278936910571F18A3691058CF4FC
:103A40008536910511F1863691053CF48F33910549
:103A5000D1F184369105E1F032C08836910591F0BC
:103A60002EC08237910541F18337910524F48037C8
:103A70009105C9F024C084379105C1F087379105BD
:103A8000C1F01DC00E94A31D20C00E9492231DC032
:103A90000E94DD1F1AC081E08093180187E29AE13D
:103AA0000E94F41C12C00E94DE190FC00E94621C0A
:103AB0000CC00E94CE1C09C00E94D71C06C082E523
:103AC0009AE10E94F41C0E94761DFF91EF91BF9134
:103AD000AF919F918F917F916F915F914F913F91A6
:103AE0002F910F900FBE0F901F90189585E69AE1C9
:103AF0000E94F41C83E89AE10E94F41C8FE99AE189
:103B00000E94F41C8EEB9AE10E94F41C8BEE9AE169
:103B10000E94F41C82E39BE10E94F41C8BE79BE172
:103B20000E94F41C82EC9BE10E94F41C83E09CE167
:103B30000E94F41C83E39CE10E94F41C84E69CE157
:103B40000E94F41C08951F93CF93DF938EB799279B
:103B5000D82FCC278DB79927C82BD92B87E69CE186
:103B60000E94F41C8EB70E9497368DB70E9497363C
:103B700080E89CE10E94F41C83E89CE10E94F41C14
:103B800012E1219688810E94973680E20E94823657
:103B90001150B9F782E99CE10E94F41C1C2F10958A
:103BA00049F0219688810E94973680E20E948236F1
:103BB0001150B9F785E99CE10E94F41C8CB10E9478
:103BC000823688E99CE10E94F41C0E94D137FFCF25
:103BD0001F920F920FB60F9211248F939F93909183
:103BE0009C00892F81548A3350F49093190180915D
:103BF0001901873421F48091130180930B019F9167
:103C00008F910F900FBE0F901F901895CF93DF9359
:103C1000EC018881882331F089910E948E36888159
:103C20008823D1F7DF91CF910895CF93DF93EC01F3
:103C3000FC018491882349F0FE0184910E948E3614
:103C40002196FE0184918823B9F7DF91CF910895E1
:103C500080919B00882324F480919C000E948236EE
:103C6000089508958091190199278734910509F4E1
:103C70005EC088349105CCF48334910509F446C0C4
:103C80008434910554F48134910541F182349105D5
:103C900044F5892B09F45CC059C085349105D9F1EC
:103CA000863491050CF03FC033C08A34910509F485
:103CB00046C08B34910544F488349105F1F1893480
:103CC000910509F440C042C08C34910599F18C34BF
:103CD0009105BCF18736910541F138C00E948A1FD9
:103CE00035C0809117018095809317010E94A81319
:103CF00080911701882319F00E94EE1827C081E0F7
:103D000090E0909303018093020120C081E01CC0E9
:103D1000109201011BC080911201809580931201C5
:103D20000E94A81313C083E00FC082E00DC00E9460
:103D3000092C08950E94852C09C086E005C087E003
:103D400003C088E001C089E080930101109219014D
:103D5000089508951F920F920FB60F9211242F937A
:103D60003F934F935F936F937F938F939F93AF9303
:103D7000BF93EF93FF931ABA87B38F7187BB14BABF
:103D80008F9880916100817E8093610012981B98CA
:103D90000E94E8138CE50E948E3682E40E948E36E3
:103DA00080E20E948E3681E20E948E3689EA9CE192
:103DB0000E94151E8CE50E948E3682E40E948E368B
:103DC00080E20E948E3683E20E948E368DEB9CE16B
:103DD0000E94151E8BEE9CE10E94F41C82E09DE186
:103DE0000E94F41C60E085E090E00E94452660E0BF
:103DF00086E090E00E94452660E087E090E00E9427
:103E0000452660E088E090E00E9445260E99FECFAE
:103E100089E29DE10E94F41C84E60E94B6360E946D
:103E20002B3CFF91EF91BF91AF919F918F917F912B
:103E30006F915F914F913F912F910F900FBE0F9017
:103E40001F901895282F84EA809374008091740045
:103E500087FFFCCF809171009927887F9070089729
:103E600019F084E690E0089586E88093730084E872
:103E7000809374008091740087FFFCCF8091710063
:103E80009927887F9070489719F085E690E008950B
:103E90002093730084E8809374008091740087FFFE
:103EA000FCCF809171009927887F9070889719F0D6
:103EB00086E690E008956093730084E88093740030
:103EC0008091740087FFFCCF809171009927887FD3
:103ED0009070889719F087E690E0089584E98093C0
:103EE000740080E090E00895089580910001882397
:103EF00081F00D9B0EC080E391E00E947435982FF5
:103F000080912001882329F4779BFECF9FB90D99DA
:103F1000F2CF08951B988CE50E948E3680E40E94B3
:103F20008E3680E20E948E3680E30E948E360E949A
:103F3000DD150E94EB150E94D13710921901809176
:103F40001901813431F00E9480238091190181345C
:103F5000D1F70E942B3C08951F93CF93DF938EB728
:103F60009927D82FCC278DB79927C82BD92B83E534
:103F70009DE10E94F41C8EB70E9497368DB70E9477
:103F800097368AE69DE10E94F41C8DE69DE10E9431
:103F9000F41C1C2F109549F0219688810E949736B9
:103FA00080E20E9482361150B9F78CE79DE10E94B1
:103FB000F41CDF91CF911F910895EF92FF920F9320
:103FC0001F93CF938FE79DE10E94F41C8FE99DE141
:103FD0000E94F41C8091840F9091850FA091860F10
:103FE000B091870F8B2F9927AA27BB270E9497365E
:103FF0008091840F9091850FA091860FB091870FCB
:10400000CD01AA27BB270E9497368091840F9091FB
:10401000850FA091860FB091870F892F9A2FAB2F14
:10402000BB270E9497368091840F9091850FA091B5
:10403000860FB091870F0E94973685EC9DE10E9414
:10404000F41C88EC9DE10E94F41C8091740F909107
:10405000750F892F99270E9497368091740F909140
:10406000750F0E94973685EF9DE10E94F41C88EF42
:104070009DE10E94F41C8091680F0E9497368CE0AD
:104080009EE10E94F41C8FE09EE10E94F41C80914E
:104090005A0F0E94973688E29EE10E94F41C8BE240
:1040A0009EE10E94F41C8091700F9091710FA0917D
:1040B000720FB091730F8B2F9927AA27BB270E94ED
:1040C00097368091700F9091710FA091720FB091FF
:1040D000730FCD01AA27BB270E9497368091700FDE
:1040E0009091710FA091720FB091730F892F9A2F39
:1040F000AB2FBB270E9497368091700F9091710F64
:10410000A091720FB091730F0E94973685E59EE1E2
:104110000E94F41C88E59EE10E94F41C8091400FEF
:104120000E9497368CE69EE10E94F41C8FE69EE189
:104130000E94F41C8FE70E9414370E94973688E88B
:104140009EE10E94F41C8BE89EE10E94F41C8FE427
:104150000E9414370E94973683EA9EE10E94F41C65
:1041600086EA9EE10E94F41C8091FA0F0E94973625
:104170008DEB9EE10E94F41C80EC9EE10E94F41CF9
:104180008091500F9091510F892F99270E94973657
:104190008091500F9091510F0E94973684ED9EE1CF
:1041A0000E94F41C87ED9EE10E94F41C80917C0F1C
:1041B00090917D0FA0917E0FB0917F0F8B2F99274B
:1041C000AA27BB270E94973680917C0F90917D0F84
:1041D000A0917E0FB0917F0FCD01AA27BB270E942F
:1041E000973680917C0F90917D0FA0917E0FB091BA
:1041F0007F0F892F9A2FAB2FBB270E949736809174
:104200007C0F90917D0FA0917E0FB0917F0F0E9447
:1042100097368BEE9EE10E94F41C8EEE9EE10E948A
:10422000F41C809100010E94973685E09FE10E9476
:10423000F41C88E09FE10E94F41C8091150190918C
:104240001601892F99270E94973680911501909128
:1042500016010E94973687E19FE10E94F41C41E01D
:104260006FE370E080E090E00E94E5378330B9F7BB
:104270008AE19FE10E94F41C8FE70E94143787FDBA
:10428000FBCFBFE0EB2EA3E0FA2EC1E087E40E9453
:104290006B378C010E94973688E49FE10E94F41CE2
:1042A000812F99270E9497368AE49FE10E94F41C8F
:1042B000C15060F78CE49FE10E94F41CFA948FEFE8
:1042C000F81619F78EE49FE10E94F41CEA948FEF30
:1042D000E816C9F681E59FE10E94F41C0E9478214E
:1042E0000E94D137CF911F910F91FF90EF900895C9
:1042F0000F931F93CF931092800F0E945439809197
:10430000680F882331F00E9454398091680F882308
:10431000D1F780E391E00E9465358FEF9FEFAFEF1B
:10432000BFE08093041090930510A0930610B09303
:1043300007108091540F9091550FA091560FB09196
:10434000570F8093640F9093650FA093660FB093FF
:10435000670F80E391E090936D0F80936C0F81E085
:104360008093800F0E9454390E9454390FC00E94DC
:1043700054398091680F882349F480E391E00E94CA
:104380003136809718F481E090E03DC080E391E001
:104390000E943136809758F384E59FE10E94F41C17
:1043A00001E013E0C3E080E391E00E9474350E94D5
:1043B000973683E89FE10E94F41CC150A0F785E87E
:1043C0009FE10E94F41C115068F787E89FE10E946A
:1043D000F41C015030F78AE89FE10E94F41C10920F
:1043E000800F0E9454398091680F882331F00E9419
:1043F00054398091680F8823D1F780E391E00E94BF
:10440000653580E090E0CF911F910F9108951F9343
:10441000CF93182FC62F8CE50E948E3682E40E941F
:104420008E3680E20E948E36115E812F0E948E367B
:10443000C150CF3F31F08DE89FE10E94151EC15061
:10444000D0F7CF911F9108950F931F93082F162F28
:104450008CE50E948E3682E40E948E36115E812F9A
:104460000E948E36015E802F0E948E361F910F9122
:104470000895AF92BF92CF92DF92EF92FF920F9387
:10448000CF93DF93EC01662329F422E8A22E26E3E2
:10449000B22E04C09EE8A92E96E3B92E7E0127E233
:1044A000C031D207C0F080E1C82E87E2D82ECE01FD
:1044B000B6010E94523CCB01062F805DF5010995A3
:1044C000802F99278C9D90018D9D300D9C9D300DE6
:1044D0001124C21BD30B38EEE31633E0F306C0F011
:1044E00008EEC02E03E0D02ECE01B6010E94523C51
:1044F000CB01062F805DF5010995802F99278C9DB2
:1045000090018D9D300D9C9D300D1124C21BD30B4D
:1045100034E6E316F10480F0CE0164E670E00E9418
:10452000523CCB01062F805DF501099584E6089F7A
:10453000C0011124C81BD90B8AE0E816F10480F0F1
:10454000CE016AE070E00E94523CCB01062F805DF4
:10455000F50109958AE0089FC0011124C81BD90BF9
:104560008C2F805DF5010995DF91CF910F91FF9020
:10457000EF90DF90CF90BF90AF900895CF93DF93EF
:104580009C01FB010E94523CEB01C901BF010E944A
:10459000523CF695E795E817F90708F42196CE0105
:1045A000DF91CF910895681718F4861B9927089515
:1045B000681B862F992708950895AF92BF92CF92D6
:1045C000DF92EF92FF920F931F93CF93DF9380912F
:1045D00013018093040185E0B82EEB2CFF24E70142
:1045E000D695DC2FCC27D795C795CE018B5C9E4FF7
:1045F0000E94353CA82E1CE0C12E11E0D12ECE0C1D
:10460000DF1CF60180818A1508F06AC08081082FBE
:104610001127000F111F0C0F1D1F095C1E4FC80131
:104620000E94353CC82FDD270F5F1F4FC8010E9435
:10463000353C9927982F8827C80FD91FF60180810C
:104640009E01369527953695279580FF0CC0AE01C3
:10465000421B530BCE01969587959E01220F331F67
:10466000280F391F08C0AE0164E0569547956A953A
:10467000E1F72C0F3D1F80911A0190911B018417C7
:10468000950740F180911A0190911B012817390775
:1046900008F18A2D99270197E701C45FDE4F288131
:1046A00033278217930791F4F694FE2CEE24F794A7
:1046B000E79486E391E0E80EF91EC7010E94353CBD
:1046C0008093190188818F5F88830FC088818F5FF5
:1046D000888306C0ECE0F1E0EE0EFF1EF7011082C9
:1046E000BA94FFEFBF1609F078CFDF91CF911F91F9
:1046F0000F91FF90EF90DF90CF90BF90AF90089513
:1047000080911301992720910401821B910903973D
:1047100044F085E0E82FFF27E45FFE4F10828150D0
:10472000C8F708950F931F93CF93DF9386EA9FE115
:104730000E94F41CC0E0D0E08D2F99270E9497368C
:104740008C2F0E94973682EC9FE10E94F41C03E0BC
:1047500013E0CE0121960E94353C0E94973685ECED
:104760009FE10E94F41C1150A0F787EC9FE10E948A
:10477000F41C015068F789EC9FE10E94F41C85E06D
:10478000C030D807C8F28CEC9FE10E94F41CDF9186
:10479000CF911F910F91089580911401992700974F
:1047A00029F0019731F40E942B2408950E94DE2302
:1047B000089580EA0E947313089508950F931F933C
:1047C000809101019927009721F08130910591F1A5
:1047D00036C084E090E00E94353C082F112783E02A
:1047E00090E00E94353C080F111D012B69F464E034
:1047F00082E00E94072261E083E00E9424228FEC85
:104800009FE10E94151E21C08CE50E948E3682E435
:104810000E948E3680E20E948E3681E20E948E36A1
:104820008AE090E20E94151E0E94B42481E08093E9
:1048300014010EC0909316018093150106C01092CA
:10484000000180E391E00E94653584E080930101DE
:104850001F910F910895CF93809101019927843082
:104860009105D1F1853091057CF481309105A1F15C
:10487000823091051CF4892BC9F048C08230910523
:1048800019F1039721F142C08730910579F1883001
:10489000910534F485309105E1F1069729F136C090
:1048A0008830910529F1099739F130C08091680F5E
:1048B000882379F580E391E00E94F735813049F54E
:1048C00082E08093010125C00E94442502C00E941D
:1048D0008325C82F882319F00E948B241AC00E94B8
:1048E000B424C093010115C061E003C061E005C0BC
:1048F00060E08AE090E003C060E084E690E00E941F
:10490000ED250E94B4241092010103C082EA0E94A6
:104910007313CF910895CF930E9431261092800F88
:104920001092000184E080930101109214018CE543
:104930000E948E3682E40E948E3680E20E948E367D
:1049400081E20E948E36C0E080E20E948E36CF5F08
:10495000C837D0F380E391E00E9465350E94D137DB
:104960000E94A715CF9108950E9431261092800FC2
:104970008091680F882331F00E9454398091680F2C
:104980008823D1F71092000180E391E00E94653501
:1049900080911501909116010E945F268530E9F4FF
:1049A0008AE390E20E94F41C809115019091160117
:1049B000892F99270E9497368091150190911601B1
:1049C0000E9497368FE690E20E94F41C81E090E00E
:1049D000909316018093150108950E9439290E9431
:1049E000C2251092800F8091680F882331F00E94B9
:1049F00054398091680F8823D1F780915C0F909192
:104A00005D0FA0915E0FB0915F0F809304109093A3
:104A10000510A0930610B09307108091780F909125
:104A2000790FA0917A0FB0917B0F8093640F9093D0
:104A3000650FA093660FB093670F80E391E09093AA
:104A40006D0F80936C0F0E94653581E08093800F1D
:104A50008091680F882349F40E9454398091680F2F
:104A60008823D1F302C00E94543980E391E00E9470
:104A7000313680549B40B8F381E0809300010E945E
:104A80003B2680E090E008950F931F9384E090E030
:104A90000E94353C9927182F002783E090E00E9460
:104AA000353CA801480F511D8091150190911601C8
:104AB0002091020130910301820F931F9093160100
:104AC000809315018091150190911601481759079F
:104AD000A8F48091150190911601841B950B909379
:104AE00016018093150180911701882339F4809174
:104AF0001201882319F481E090E002C080E090E088
:104B00001F910F9108950F931F9384E090E00E94EE
:104B1000353C9927182F002783E090E00E94353C10
:104B2000A801480F511D2091150130911601809167
:104B30000201909103018217930778F48091150187
:104B4000909116012091020130910301821B930B79
:104B5000909316018093150110C0809102019091ED
:104B600003012091150130911601821B930B481B04
:104B7000590B509316014093150180E090E01F916E
:104B80000F910895CF938CE50E948E3682E40E94A7
:104B90008E3680E20E948E3682E20E948E36C0E01F
:104BA00080E20E948E36CF5FC036D0F31092F10FB4
:104BB00084E00E94982A8CE50E948E3682E40E944E
:104BC0008E3680E20E948E3682E20E948E3681E925
:104BD0009FE00E94061ECF9108950F931F93CF93DD
:104BE000DF93EC01662321F184E090E00E94353CE4
:104BF0009927182F002783E090E00E94353C980108
:104C0000280F311D80911501909116018C0F9D1F69
:104C100090931601809315018091150190911601D2
:104C200028173907C8F4309316012093150114C0D2
:104C30008091150190911601C817D90738F4809119
:104C40001501909116018C1B9D0B02C081E090E034
:104C50009093160180931501DF91CF911F910F91D1
:104C6000089561E084E10E94221F882319F0865F85
:104C70000E947313089560E084E10E94221F88233C
:104C800019F0825E0E94731308959C01E199FECF92
:104C9000832F99278FBB2EBB6DBB84E08CBB86E036
:104CA0008CBB08959C0142B78CB59927982F882713
:104CB000840F911DB9010E94523C019608953F92C4
:104CC0004F925F926F927F928F929F92AF92BF921C
:104CD000CF92DF92EF92FF920F931F93CF93DF93C8
:104CE0003C01892B09F49BC184E090E00E94353C93
:104CF0009927182F002783E090E00E94353C080F89
:104D0000111D0615170508F48AC110920001430110
:104D10000894810891088114910419F451E0852EBA
:104D2000912CC7E3D1E00FEF1FE78016910698F4AE
:104D30002897CE0121960E94353C082F1127CE01DD
:104D400021960E94353C9927982F8827080F191F14
:104D50008016910668F3CE0121960E94353C992772
:104D6000AA27BB278093840F9093850FA093860F6B
:104D7000B093870FCE0121960E94353C9927AA2730
:104D8000BB272227382F492F5A2F8091840F9091CB
:104D9000850FA091860FB091870F820F931FA41FDC
:104DA000B51F8093840F9093850FA093860FB093C7
:104DB000870FCE0121960E94353C9927AA27BB2751
:104DC000AC01332722278091840F9091850FA09109
:104DD000860FB091870F820F931FA41FB51F80937A
:104DE000840F9093850FA093860FB093870FCE0109
:104DF0000E94353C9927AA27BB27582F44273327E1
:104E000022278091840F9091850FA091860FB091F9
:104E1000870F820F931FA41FB51F8093840F909359
:104E2000850FA093860FB093870F8091840F909188
:104E3000850FA091860FB091870F80930501909305
:104E40000601A0930701B093080168010894C10806
:104E5000D1081092800F0E9454398091680F8823E6
:104E600031F00E9454398091680F8823D1F780E394
:104E700091E00E9465358FEF9FEFAFEFBFE0809329
:104E8000041090930510A0930610B0930710809122
:104E9000840F9091850FA091860FB091870F80931A
:104EA000640F9093650FA093660FB093670F80E334
:104EB00091E090936D0F80936C0F82E08093800F50
:104EC0000E9454390E9454398091FA0F9927982FE3
:104ED0008827990F9093750F8093740FC614D70489
:104EE00008F0B1C1C4010197C816D90681F48091B8
:104EF000840F9091850FA091860FB091870F8093BA
:104F0000050190930601A0930701B09308018091D9
:104F1000FA0F9927982F8827990F2091740F3091B5
:104F2000750F2817390709F061C00DC00E94543968
:104F30008091680F882339F480E391E00E94313634
:104F4000049708F46CC080E391E00E943136049726
:104F500068F380E391E00E947435E82EFF24002777
:104F6000112780E391E00E9474359927AA27BB2777
:104F7000BA2FA92F982F8827E80EF91E0A1F1B1F8A
:104F800080E391E00E9474359927AA27BB27DC01B2
:104F900099278827E80EF91E0A1F1B1F80E391E05E
:104FA0000E9474359927AA27BB27B82FAA279927CB
:104FB0008827E80EF91E0A1F1B1FE092840FF0924B
:104FC000850F0093860F1093870F1092750F109224
:104FD000740F0CC00E9454398091680F882331F4FB
:104FE00080E391E00E9431368097C8F080E391E041
:104FF0000E943136809770F380E391E00E9474350F
:10500000B82E882379F48093800F8091680F8823CD
:1050100031F00E9454398091680F8823D1F785E0E0
:1050200090E015C18CE08093900FB092910F80E3D7
:1050300091E00E9474358093920F80E391E00E948A
:1050400074358093930F80E391E00E9474358093D0
:10505000940F80E391E00E9474358093950F80E374
:1050600091E00E9474358093960F80E391E00E9456
:1050700074358093970F80E391E00E94743580939C
:10508000980F80E391E00E947435482E80E391E010
:105090000E947435582E80E391E00E947435A82E4A
:1050A0008EE28093990F40929A0F50929B0FA0929C
:1050B0009C0F10929D0F80E391E00E947435382E72
:1050C000C8E080E391E00E947435C150D1F780E3DD
:1050D00091E00E9474359927AA27BB278C01FF24F1
:1050E000EE2480E391E00E9474359927AA27BB271C
:1050F000B82FAA2799278827E80EF91E0A1F1B1F19
:10510000E092780FF092790F00937A0F10937B0F53
:1051100080E391E00E94743580E391E00E94743551
:1051200080E391E00E94743580E391E00E94743541
:1051300080E391E00E947435E82EFF2400271127B8
:1051400080E391E00E9474359927AA27BB27BA2FE4
:10515000A92F982F8827E80EF91E0A1F1B1F809180
:10516000780F9091790FA0917A0FB0917B0F8E0DEF
:105170009F1DA01FB11F8093780F9093790FA0936C
:105180007A0FB0937B0F80E391E00E947435E82E94
:10519000FF240027112780E391E00E9474359927AE
:1051A000AA27BB27BA2FA92F982F8827E80EF91E08
:1051B0000A1F1B1F80E391E00E9474359927AA27DC
:1051C000BB27DC0199278827E80EF91E0A1F1B1F41
:1051D00080E391E00E9474359927AA27BB27B82F56
:1051E000AA2799278827E80EF91E0A1F1B1FE0929D
:1051F0005C0FF0925D0F00935E0F10935F0F85EED2
:10520000B81691F08DE4481679F480E5581661F4EB
:1052100083E3A81649F4832D99278E719070892B0A
:1052200019F40894C11CD11C8091740F9091750FD2
:1052300080969093750F8093740F0E945439C61412
:10524000D70408F44FCE1092800F87E090E0DF91F2
:10525000CF911F910F91FF90EF90DF90CF90BF9073
:10526000AF909F908F907F906F905F904F903F9006
:105270000895CF92DF92EF92FF920F931F93CF93F7
:10528000DF93CDB7DEB72F970FB6F894DEBF0FBE12
:10529000CDBF0091740F1091750F005210402091F6
:1052A000050130910601409107015091080180915C
:1052B000840F9091850FA091860FB091870F2817CA
:1052C00039074A075B0741F08091FA0F9927982F19
:1052D0008827990F080F191F1092800F8091680F6F
:1052E000882331F00E9454398091680F8823D1F7C8
:1052F000C801AA27BB278093041090930510A093A0
:105300000610B09307108091050190910601A091BD
:105310000701B09108018093640F9093650FA093EB
:10532000660FB093670F80E391E090936D0F8093C9
:105330006C0F0E94653581E08093800F0E94543984
:10534000EE24FF248EE00730180730F0FAEFEF2E3E
:10535000F1EFFF2EE00EF11E8091680F8823A1F07F
:105360000E945439E114F10459F080E391E00E9465
:10537000743580912001882319F40894E108F1081C
:105380008091680F882361F7E8E0CE2ED12C1F862C
:1053900080E391E00E94A23580E391E00E94A23573
:1053A0008E8780E391E00E94A23580E391E00E9425
:1053B000A2358D8780E391E00E94A23580E391E0E1
:1053C0000E94A23580E391E00E94A23580E391E043
:1053D0000E94A2358C8780E391E00E94A23580E391
:1053E00091E00E94A2358B8780E391E00E94A23574
:1053F00080E391E00E94A2358A8780E391E00E94D9
:10540000A23580E391E00E94A235898780E391E094
:105410000E94A23580E391E00E94A235888780E354
:1054200091E00E94A23580E391E00E94A2358F8333
:1054300080E391E00E94A23580E391E00E94A235D2
:1054400080E391E00E94A235182F80E391E00E9452
:10545000A23580E391E00E94A2358E8380E391E043
:105460000E94A23580E391E00E94A2358D8380E303
:1054700091E00E94A23580E391E00E94A2358C83E6
:1054800080E391E00E94A23580E391E00E94A23582
:105490008B8380E391E00E94A23580E391E00E943B
:1054A000A2358A8380E391E00E94A2358983812F0F
:1054B00099278F7090700F9761F5E8E0CE16D104B0
:1054C00011F41092900F71E0E72EF12C9091900F53
:1054D00021E93FE0A901490F511DDE01AE0DBF1DBD
:1054E00011968C91FA0180830894E11CF11C2F5FC6
:1054F0003F4F882379F79E0D92509093900F8981AA
:1055000086FD07C00894C108D108C114D10409F070
:105510003ECF2F960FB6F894DEBF0FBECDBFDF9102
:10552000CF911F910F91FF90EF90DF90CF90089552
:10553000FF920F931F93CF93482F01E91FE0FF24A1
:105540008091910F882339F0F3940F5F1F4FF8017A
:1055500080818823C9F780E68F19F82E442371F0E3
:1055600080E690E08F199109242F332728173907F7
:105570002CF4021B130BF8011082F40E8091910F92
:10558000803249F481E99FE00E94002CF3948091DD
:10559000910F8032B9F3FF2009F44FC08091A80F1A
:1055A00099278D32910509F448C08E32910524F473
:1055B000809709F442C00BC08E9749F460E288EAF4
:1055C0009FE00E94EA2BFA9438C0C92F25C080E6DC
:1055D00090E08F19910949970CF4F7C08091A90FB9
:1055E000803259F18091A90F8D3239F18091A90F44
:1055F0008E3219F1C1E0E7EAFFE08081803261F08C
:1056000080818D3249F080819C2F9F5F8E32E9F23C
:10561000C92F3197983188F3C73178F4FC1668F0B8
:10562000FC1A09EA1FE00C1B1109CC2331F060E2DF
:10563000C8010E94EA2BC150D1F78091A90F803296
:1056400049F489EA9FE00E94002CF3948091A90F0D
:105650008032B9F3FF2009F44FC08091C00F992721
:105660008D32910509F448C08E32910524F480975B
:1056700009F442C00BC08E9749F460E280EC9FE0D1
:105680000E94EA2BFA9438C0C92F25C080E690E02A
:105690008F199109C1970CF498C08091C10F803285
:1056A00059F18091C10F8D3239F18091C10F8E3245
:1056B00019F1C1E0EFEBFFE08081803261F0808181
:1056C0008D3249F080819C2F9F5F8E32E9F2C92F85
:1056D0003197983188F3C73178F4FC1668F0FC1ADA
:1056E00001EC1FE00C1B1109CC2331F060E2C80172
:1056F0000E94EA2BC150D1F78091C10F803249F44A
:1057000081EC9FE00E94002CF3948091C10F8032C5
:10571000B9F3FF2009F44DC08091D80F99278D323D
:10572000910509F446C08E32910524F4809709F45E
:1057300040C00AC08E9741F460E288ED9FE00E946D
:10574000EA2B37C0C92F25C080E690E08F19910958
:1057500089349105D4F18091D90F803251F1809133
:10576000D90F8D3231F18091D90F8E3211F1C1E014
:10577000E7EDFFE08081803261F080818D3249F079
:1057800080819C2F9F5F8E32E9F2C92F319798312B
:1057900088F3C73170F4FC1660F009ED1FE00C1BB4
:1057A0001109CC2331F060E2C8010E94EA2BC150FC
:1057B000D1F78091D90F803241F489ED9FE00E94AA
:1057C000002C8091D90F8032C1F3CF911F910F919E
:1057D000FF9008959C01FC018081882321F031967F
:1057E00080818823E1F7E217F30731F0808181831C
:1057F0003197E217F307D1F78081818360830895A1
:10580000FC018081882321F0818181938823E1F745
:1058100008950F931F930E9431261092800F85E008
:105820008093010180911701882309F06BC080915A
:105830001301282F332780910B01281B31092A30AF
:10584000310509F05FC08091130180930B018091B5
:1058500002019091030182339105C1F083339105D8
:1058600030F48130910551F00A9769F018C0843600
:10587000910579F0845F914079F011C03093030174
:105880002093020112C082E390E00BC084E690E016
:1058900008C084EF91E005C088EE93E002C081E08B
:1058A00090E0909303018093020184E090E00E94D5
:1058B000353C9927182F002783E090E00E94353C63
:1058C000080F111D8091020190910301801791072B
:1058D00030F081E090E0909303018093020164E056
:1058E00083E00E94072261E084E00E94242282E794
:1058F00090E20E94151E61E08091020190910301E7
:105900000E9439221F910F910895CF93DF93109237
:1059100019010E948B2461E0862F0E9424228FE7C8
:1059200090E20E94151ECAE6D1E166E083E00E9483
:10593000072261E084E00E942422FE0134968591D2
:1059400094910E94151E809119018C3409F441C074
:105950008091190199278834910581F08934910546
:1059600024F48134910529F02FC08B349105C9F0BE
:105970002BC0109219010E948A1F26C01092190193
:1059800065E083E00E940722FE013296C591D49122
:1059900061E084E00E942422FE0134968591949176
:1059A00011C01092190165E083E00E940722FE01F8
:1059B000C591D49161E084E00E942422FE013496D6
:1059C000859194910E94151E809119018C3409F0E3
:1059D000BFCF1092190168E081E00E940722FE010A
:1059E000369685919491FC01099568E081E00E94CA
:1059F00007220E94C9150E94A7150E94A813DF91D3
:105A0000CF9108950895CF9361E0862F0E942422BC
:105A100087EB90E20E94151E80E090E00E94353CEA
:105A2000C82FC0956BE085E00E9424228C2F992717
:105A300061E00E943922809119018C3489F18091B2
:105A4000190199278834910581F08934910524F44E
:105A50008134910529F020C08B34910561F01CC080
:105A6000109219010E948A1F17C010921901CF3F8E
:105A700031F0CF5F04C010921901C111C15061E033
:105A800085E00E9407226BE085E00E9424228C2F93
:105A9000992761E00E943922809119018C3479F6AE
:105AA000C0956C2F80E090E00E9445266C2F86E424
:105AB0000E94221F882319F088580E94731381E0E6
:105AC0000E94B6366C2F88E40E94221F882319F0AA
:105AD0008E570E947313CF910895CF9361E0862F64
:105AE0000E94242281E091E20E94151E81E090E054
:105AF0000E94353CC82F6BE085E00E9424228C2F49
:105B00000E942D2E809119018C3491F18091190100
:105B100099278834910581F08934910524F48134E2
:105B2000910529F021C08B34910569F01DC01092B8
:105B300019010E948A1F18C010921901CF5FCD3041
:105B400041F4CCE006C010921901C150C33F09F4E2
:105B5000C4EF61E085E00E9407226BE085E00E94CF
:105B600024228C2F0E942D2E809119018C3471F6E5
:105B70006C2F81E090E00E9445266C2F8CE70E94FC
:105B8000221F882319F082590E94731381E00E941A
:105B9000B6360E94EB2ECF910895CF9361E0862F09
:105BA0000E9424228AE491E20E94151E82E090E085
:105BB0000E94353CC82F6BE085E00E9424228C2F88
:105BC0000E942D2E809119018C3491F18091190140
:105BD00099278834910581F08934910524F4813422
:105BE000910529F021C08B34910569F01DC01092F8
:105BF00019010E948A1F18C010921901CF5FCD3081
:105C000041F4CCE006C010921901C150C33F09F421
:105C1000C4EF61E085E00E9407226BE085E00E940E
:105C200024228C2F0E942D2E809119018C3471F624
:105C30006C2F82E090E00E9445266C2F8BE70E943B
:105C4000221F882319F088580E94731381E00E9454
:105C5000B6360E94EB2ECF91089599278C3091058E
:105C600009F4B3C08D309105A4F58530910509F490
:105C700097C086309105B4F48230910509F487C04D
:105C8000833091053CF4009709F47BC0019709F437
:105C90007BC09EC08330910509F47CC0049709F451
:105CA0007CC096C08830910509F483C08930910585
:105CB00044F48630910509F476C0079709F476C05C
:105CC00087C08A30910509F47AC00B970CF07AC02E
:105CD00073C0893F910509F43FC08A3F9105A4F440
:105CE000863F910581F1873F91053CF4843F910502
:105CF00011F1853F910511F16BC0873F910531F19D
:105D0000883F910531F164C08C3F910571F18D3F61
:105D100091053CF48A3F910511F18B3F910511F1FA
:105D200057C08E3F910539F18E3F91050CF18F3FA1
:105D3000910521F14DC083E991E202C08AE991E227
:105D40000E94151E089583EA91E2FACF8AEA91E251
:105D5000F7CF83EB91E2F4CF8AEB91E2F1CF83ECC2
:105D600091E2EECF89EC91E2EBCF81ED91E2E8CFC9
:105D700087ED91E2E5CF8FED91E2E2CF85EE91E202
:105D8000DFCF8DEE91E2DCCF82EF91E2D9CF8AEFC7
:105D900091E2D6CF80E092E2D3CF88E092E2D0CFFA
:105DA0008EE092E2CDCF86E192E2CACF8CE192E220
:105DB000C7CF85E292E2C4CF8CE292E2C1CF85E305
:105DC00092E2BECF8CE392E2BBCF85E492E2B8CF01
:105DD0008CE492E2B5CFCF93C0E081E090E00E94E6
:105DE000353C87FD05C081E090E00E94353CC82F1E
:105DF00082E090E00E94353C87FD05C082E090E0A3
:105E00000E94353CC80FCD3008F0CCE06C2F8DE7F8
:105E10000E94221F81E00E94B636CF9108950F9311
:105E20001F9361E0862F0E9424228AE592E20E945D
:105E3000151E0E94D1320E94B33761E083E00E94B8
:105E4000242281E99FE00E94061E61E085E00E9415
:105E5000242284E892E20E94151E84E090E00E94D1
:105E6000353C9927182F002783E090E00E94353CAD
:105E7000080F111D61E0C8010E94392261E087E02E
:105E80000E94242289E892E20E94151E8091190145
:105E90008C34E1F7109219011F910F9108951F930F
:105EA000CF93DF9361E0862F0E9424228FE992E254
:105EB0000E94151E81E090E00E947130882399F0C5
:105EC00063E082E00E94072261E083E00E942422D6
:105ED0008DEC92E20E94151E809119018C34E1F73D
:105EE00010921901C8C0182F0E94D13262E083E0DD
:105EF0000E94072261E083E00E94242281E99FE062
:105F00000E94061EC1E0D0E0CE010E9471300E94C6
:105F10004130809119018C3479F1809119019927D0
:105F20008834910581F08934910524F481349105F8
:105F300029F01EC08B34910569F01AC01092190126
:105F40000E948A1F15C010921901219761F4C1E0C7
:105F5000D0E009C0109219012196CE010E94713043
:105F6000882321F02197CE010E9471300E94413098
:105F7000809119018C3489F6109219012091540FE7
:105F80003091550F4091560F5091570F8091780FD7
:105F90009091790FA0917A0FB0917B0F2817390754
:105FA0004A075B0709F411E08091780F9091790F0F
:105FB000A0917A0FB0917B0F8093540F9093550F5F
:105FC000A093560FB093570F112309F48DCF8091F2
:105FD000540F9091550FA091560FB091570F682F05
:105FE00085E090E00E9445268091540F9091550FD6
:105FF000A091560FB091570F892F9A2FAB2FBB2727
:10600000682F86E090E00E9445268091540F909181
:10601000550FA091560FB091570FCD01AA27BB275E
:10602000682F87E090E00E9445268091540F909160
:10603000550FA091560FB091570F8B2F9927AA2774
:10604000BB27682F88E090E00E94452664E0862FF9
:106050000E9407220E94F6150E94CF168091170118
:10606000882319F00E94EE1806C081E090E090931A
:106070001601809315010E94B337DF91CF911F91D4
:10608000089548E050E06CEF72E281E99FE00E94E1
:10609000443C892B19F465E073E20CC048E050E001
:1060A0006CE173E281E99FE00E94443C892B39F462
:1060B00065E273E281E99FE00E943D3C02C00E94DC
:1060C000392980E00E94982A63E085E00E94072237
:1060D00061E085E00E94242281E99FE00E94061E83
:1060E00008956F927F928F929F92AF92BF92CF92BC
:1060F000DF92EF92FF920F931F93CF936C01892B46
:1061000019F481E090E01BC28091540F9091550FDB
:10611000A091560FB091570F0297A105B10581F4D8
:1061200081E0C816D10449F40E94AD3206C282E073
:1061300090E005C284E090E002C20894C108D10852
:1061400046010894810891088114910419F481E0B2
:10615000882E912C109200011092800F0E945439C9
:106160008091680F882331F00E9454398091680F24
:106170008823D1F780E391E00E9465358091540F28
:106180009091550FA091560FB091570F8093840FA7
:106190009093850FA093860FB093870F8FEF9FEF9B
:1061A000AFEFBFE08093041090930510A09306100A
:1061B000B09307108091840F9091850FA091860F66
:1061C000B091870F8093640F9093650FA093660F33
:1061D000B093670F80E391E090936D0F80936C0F05
:1061E00082E08093800F0E9454390E94543980913C
:1061F000FA0F9927982F8827990F9093750F8093FE
:10620000740F662477246C147D0408F064C1C40103
:1062100001976816790681F48091840F9091850F1B
:10622000A091860FB091870F80930501909306018E
:10623000A0930701B09308018091FA0F9927982F36
:106240008827990F2091740F3091750F28173907FF
:1062500009F062C00DC00E9454398091680F8823F4
:1062600039F480E391E00E943136049708F45FCF5F
:1062700080E391E00E943136049768F380E391E077
:106280000E947435E82EFF240027112780E391E057
:106290000E9474359927AA27BB27BA2FA92F982FB8
:1062A0008827E80EF91E0A1F1B1F80E391E00E9459
:1062B00074359927AA27BB27DC0199278827E80E80
:1062C000F91E0A1F1B1F80E391E00E947435992775
:1062D000AA27BB27B82FAA2799278827E80EF91ED7
:1062E0000A1F1B1FE092840FF092850F0093860F08
:1062F0001093870F1092750F1092740F0DC00E94AB
:1063000054398091680F882339F480E391E00E942A
:106310003136809708F40ECF80E391E00E94313649
:10632000809768F380E391E00E947435B82E88234B
:1063300079F48093800F8091680F882331F00E9458
:1063400054398091680F8823D1F788E090E0F7C036
:106350008CE08093900FB092910F80E391E00E94C7
:1063600074358093920F80E391E00E94743580939E
:10637000930F80E391E00E9474358093940F80E343
:1063800091E00E9474358093950F80E391E00E9424
:1063900074358093960F80E391E00E94743580936A
:1063A000970F80E391E00E9474358093980F8EE2FE
:1063B0008093990F80E391E00E94743580939A0F47
:1063C00080E391E00E94743580939B0F80E391E01D
:1063D0000E94743580939C0F10929D0F80E391E092
:1063E0000E947435A82EC8E080E391E00E947435C5
:1063F000C150D1F780E391E00E9474359927AA2714
:10640000BB278C01FF24EE2480E391E00E947435C9
:106410009927AA27BB27B82FAA2799278827E80EEC
:10642000F91E0A1F1B1FE092780FF092790F00935C
:106430007A0F10937B0FC4E080E391E00E947435E3
:10644000C150D1F780E391E00E947435E82EFF241B
:106450000027112780E391E00E9474359927AA272D
:10646000BB27BA2FA92F982F8827E80EF91E0A1FDD
:106470001B1F8091780F9091790FA0917A0FB091A6
:106480007B0F8E0D9F1DA01FB11F8093780F9093DF
:10649000790FA0937A0FB0937B0FC4E080E391E073
:1064A0000E947435C150D1F785EEB81629F0A4FECC
:1064B00003C00894611C711C8091740F9091750F3A
:1064C00080969093750F8093740F0E9454396C14CA
:1064D0007D0408F49CCE1092800F8091780F9091EB
:1064E000790FA0917A0FB0917B0F0097A105B105AC
:1064F00061F482E090E0A0E0B0E08093780F9093A8
:10650000790FA0937A0FB0937B0F80910501909142
:106510000601A0910701B09108010097A105B105FE
:1065200061F482E090E0A0E0B0E0809305019093F8
:106530000601A0930701B093080180E090E0CF919D
:106540001F910F91FF90EF90DF90CF90BF90AF9091
:106550009F908F907F906F90089582E090E0A0E0F0
:10656000B0E08093780F9093790FA0937A0FB09357
:106570007B0F8093050190930601A0930701B093D0
:1065800008016BE373E281E99FE00E943D3C8CE0EF
:106590008093900F80E290E09093750F8093740F3A
:1065A0000895EF92FF920F931F93CF93DF93809103
:1065B000540F9091550FA091560FB091570F02971D
:1065C000A105B10539F468E473E281E99FE00E9416
:1065D0003D3C39C0E090540FF090550F0091560F9C
:1065E0001091570F82E090E00E9471308091780FF7
:1065F0009091790FA0917A0FB0917B0F8093540FF7
:106600009093550FA093560FB093570FC1E0D0E071
:10661000CE0121960E9471308091780F9091790F70
:10662000A0917A0FB0917B0F8E159F05A007B1073F
:1066300079F70E943929E092540FF092550F009398
:10664000560F1093570FDF91CF911F910F91FF902D
:10665000EF9008951F93CF93DF9311E061E0862FB1
:106660000E94242287E593E20E94151EC0E0D2E139
:1066700061E084E00E942422FE0134968591949189
:106680000E94151E809119018C3409F441C080913B
:10669000190199278834910581F08934910524F4F2
:1066A0008134910529F02FC08B349105C9F02BC09E
:1066B000109219010E948A1F26C01092190162E0EF
:1066C00084E00E940722FE013296C591D49161E0D8
:1066D00084E00E942422FE0134968591949111C099
:1066E0001092190162E084E00E940722FE01C59128
:1066F000D49161E084E00E942422FE0134968591C9
:1067000094910E94151E809119018C3409F0BFCF1D
:106710001092190168E081E00E94072261E0862F53
:106720000E94242286E893E20E94151EFE013696FE
:10673000859194910E94D03368E081E00E94072205
:1067400061E0862F0E94242285EE93E20E94151EAE
:1067500061E083E00E94242287EF93E20E94151EED
:1067600061E086E00E94242281E294E20E94151EEC
:1067700010921901809119018823E1F38091190188
:106780008C3409F010E01092190168E081E00E9459
:106790000722112309F062CFDF91CF911F91089555
:1067A0008F929F92AF92BF92CF92DF92EF92FF9221
:1067B0000F931F93CF93DF935C0180917D008F7DBA
:1067C00080937D0084E880938A0080917C008062C1
:1067D00080937C00AAE3EA2EA1E0FA2E80917C004F
:1067E00085FFFCCF109289001092880080918A006A
:1067F00090E4892780938A0080E280937C00209136
:10680000130188249924809113019927422F552739
:10681000841B950B029764F580917C0085FFFCCF6B
:10682000109289001092880080918A0090E4892754
:1068300080938A0020918000809181009927982F71
:106840008827820F911DF701819391937F0108940E
:10685000811C911CF9EC8F16910450F480E2809316
:106860007C00809113019927841B950B0297A4F259
:106870002AE08216910408F4DFC000913E011091D5
:106880003F01E0E4EE2EE1E0FE2E6801E4012597F1
:106890009E01F701808191818017910710F46801B2
:1068A0008C0182E090E0E80EF91E21979FEFCF3F28
:1068B000D90779F7C0E0D0E07EE3E72E71E0F72E4C
:1068C0008E01CE01A60156954795B601640F751F3E
:1068D000E9012F5F3F4FC9F0F70120813181421755
:1068E000530738F42617370720F4820F931F0F5FE2
:1068F0001F4F22E030E0E20EF31E21973FEFCF3F23
:10690000D30719F00830110538F30115110521F0EE
:10691000B8010E94BE226C015EE3E52E51E0F52E27
:1069200002E010E0E401229702C00F5F1F4F2197A1
:106930008FEFCF3FD80749F0F701819191917F0107
:10694000B6010E94BE22409780F30034110510F07A
:106950000FE310E0809118018823F1F188E394E2BD
:106960000E94F41C88E594E20E94F41C60E0C401DB
:106970000E94392280E794E20E94F41C60E0C60184
:106980000E9439228CE894E20E94F41C60E0C80165
:106990000E94392281EB94E20E94F41C4AE3E42E27
:1069A00041E0F42EE4012197FFEFCF3FDF0781F0B4
:1069B000F701819191917F0160E00E94392284EB7F
:1069C00094E20E94F41C2197FFEFCF3FDF0781F78D
:1069D00087EB94E20E94F41CC5010894A11CB11C31
:1069E000602F0E9445260894A11CB11C3AE3E32EB7
:1069F00031E0F32E015010402FEF0F3F1207E1F06E
:106A0000C5010894A11CB11CF70160810E944526B4
:106A1000F701819191917F01892F99279501089420
:106A2000A11CB11C682FC9010E94452601501040CD
:106A3000FFEF0F3F1F0721F7C5E0D0E0E1E1F1E0F4
:106A40001082219731972FEFCF3FD207C9F780E30C
:106A500091E00E94653584E880938A0080917D00F2
:106A6000806280937D00DF91CF911F910F91FF9005
:106A7000EF90DF90CF90BF90AF909F908F90089550
:106A8000479A0895FF93EF930F93E0E3F1E001E05D
:106A9000019306E3019301E0019306E301930FE004
:106AA000019300E40083E0E3F1E001E0019306E3F9
:106AB000019301E0019306E301930FE0019300E4E9
:106AC00000830F91EF91FF9108950F93EF93FF9340
:106AD000E82FF92F04D0FF91EF910F9108950081D5
:106AE00002830181038308950F932F933F93AF9304
:106AF000BF93EF93FF93E82FF92F0BD0832F2093B1
:106B00002001FF91EF91BF91AF913F912F910F9194
:106B10000895B081A18103810A1B29F402810B1B16
:106B200011F421E008953C91119605810A1B31F47E
:106B300004810B1B19F4BF2FAE2F1696B083A183CF
:106B400020E008952F933F93AF93BF93EF93FF936C
:106B5000E82FF92F0AD0832F20932001FF91EF9186
:106B6000BF91AF913F912F910895B281A38121816F
:106B70002A1729F420812B1711F421E00895119789
:106B80003596AE1739F4BF1729F43597B481A5812E
:106B9000119735963597B283A3833C9120E00895F1
:106BA000B281A381119605810A1B31F404810B1B6C
:106BB00019F4BF2FAE2F169601810A1B89F40081AC
:106BC0000B1B71F421E50E94893627E50E94893666
:106BD00021E50E94893626E40E94893622E0089544
:106BE000D281C3812883B283A38320E008950F93C9
:106BF0002F93AF93BF93EF93FF93E82FF92F08D014
:106C0000822FFF91EF91BF91AF912F910F91089536
:106C1000B081A18103810A1B31F402810B1B19F49D
:106C200001E0202F089503E0202F089510800180B7
:106C3000328023802014310448F40218130801E044
:106C4000001A00E0100A212D302D0895248135818D
:106C50003E1B2F0B37502040300D211D32192309C8
:106C600008950F921F922F923F920F93EF93FF93ED
:106C7000E82FF92F0AD0922F832FFF91EF910F91D8
:106C80003F902F901F900F900895D0DF14800580C3
:106C90000E1A1F0A07E0001A00E0100A031A120A6F
:106CA000302D212D0895E0E3F1E001D0089531DF8A
:106CB000213009F40895232F43D020E22AD04FE059
:106CC00028DF213031F0232F3BD020E222D04A951B
:106CD000B9F72DE01ED02AE01CD00895E299FECF2E
:106CE0009FBB8EBBE09A8DB308950F9303E309B960
:106CF00008E90AB903E30093990008E900939A00B0
:106D00000F9108952F930F93282F03D00F912F9158
:106D100008950BB105FFFDCF2CB908950F93009195
:106D20009B0005FFFCCF80939C000F9108952F934B
:106D30000F931F93282F04D01F910F912F91089527
:106D40001F93122F22952F7000E3200F2A3312F089
:106D500007E0200FDEDF212F2F7000E3200F2A3302
:106D600012F007E0200FD5DF1F910895882379F0F6
:106D70000F931F938F9300EA19E100001A95E9F72A
:106D80000A95D1F78A95B9F78F911F910F910895C0
:106D90000F931F930EE3009362000EE300936100D4
:106DA00097988F9A00EE08BB00EF07BB00E00ABB84
:106DB00004BB10E000E00000000000000000000044
:106DC00000000000000000000000000000000000C3
:106DD0000000000000000000000000000A9559F7C4
:106DE0001A9541F7979A10E000E0000000000000BB
:106DF0000000000000000000000000000000000093
:106E00000000000000000000000000000000000082
:106E10000A9559F71A9541F7E0E4FFE000E0008396
:106E200011241F910F9108952F93282F03D0822FA3
:106E30002F9108950F9308B323FB05F924FB06F95E
:106E400025FB07F908BB0091620026FB02F927FB2E
:106E500003F900936200009162000F7E00936200CC
:106E60000000000000000000000029B30091620053
:106E70000061009362000F9108950F932F933F9349
:106E8000282F362F04D03F912F910F91089508B3EA
:106E900023FB05F924FB06F925FB07F908BB009144
:106EA000620026FB02F927FB03F9009362000091C0
:106EB00062000D7F009362003BBB0FEF0ABB000036
:106EC0000000000000000091620002600093620078
:106ED00000E00ABB08952F933F93282F05D0822FFF
:106EE000932F3F912F9108950F9308B323FB05F93A
:106EF00024FB06F925FB07F908BB0091620026FB7D
:106F000002F927FB03F900936200009162000F7EF3
:106F1000009362000000000029B333B300916200C7
:106F20000061009362000F9108950E94A03620E254
:106F30000E94893629E40E94893624E40E94893619
:106F400025E40E94893622E70E94893621E30E94C7
:106F5000893626E30E9489362DE00E9489362AE090
:106F60000E948936C2CF0F932F933F930FE7202FB4
:106F700061DF27FDFBCF26FFF9CF07E5202F0DE0CE
:106F8000302F85DF0FE7202F55DF26FFFBCF0FE7E0
:106F9000202F02EE302F7BDF11243F912F910F9194
:106FA00008950F932F933F930FE7202F43DF27FD83
:106FB000FBCF26FFF9CF0FE7202F00EE302F67DF42
:106FC00011243F912F910F9108950F932F933F9389
:106FD000EF93FF93242F9F938F937F936F930BD007
:106FE0006F917F918F919F91822FFF91EF913F91B0
:106FF0002F910F910895E0E4FFE00081013031F11D
:107000002F932FE717DF27FD02C026FD03C02F9126
:1070100022E008953F9127E53ADFEDB7FEB73396BA
:107020002FE5319134DF27E6319131DF2FE63191C1
:107030002EDF27E73191306E2ADF2FE730E227DF9E
:10704000E0E4FFE001E0008322E00895322F2FE723
:10705000F1DE27FD09C020FD0FC024FF05C026FF7B
:1070600003C022FD09C002C022E00895E0E4FFE071
:1070700000E0008323E008950E94A03620E20E94F1
:107080008936232F0E94A03620E20E948936EDB770
:10709000FEB7379622910E94A03622910E94A03618
:1070A00022910E94A03622910E94A03620E20E94E6
:1070B000893623E50E94893625E60E94893625E631
:1070C0000E9489362BE60E94893623E50E94893684
:1070D00025E60E94893623E60E94893624E70E942D
:1070E00089362FE60E94893622E70E9489362DE0F4
:1070F0000E9489362AE00E9489362FE49BDE00E058
:107100000093400F22E008952FE794DE27FDFCCF87
:107110002DE0FFDD2AE0FDDD2AE0FBDD04E1E02ECD
:1071200008E0F02E27E4E0DE0BDE20E2F2DD232F84
:1071300007DE20E2EEDDFA94A9F72DE0EADD2AE091
:10714000E8DDEA9469F708950F93EF93FF93EAE57A
:10715000FFE000E0008300270093600F0093610FC1
:107160000093620F0093630F0093FC0F0093FD0FD9
:107170000093FE0F0093FF0FE8E6FFE000E00083BE
:10718000E0E8FFE000E00083FF91EF910F910895A8
:107190000F932F933F93EF93FF930F921F922F9292
:1071A0003F924F920091400F003021F00E94FB3738
:1071B0000C94D23800E00F930F930F930FE30F93CB
:1071C00021E019DF0F910F910F910F9103E020172C
:1071D00089F727E40E94743727E40E94743727E474
:1071E0000E94743727E40E94743727E40E947437A2
:1071F00027E40E94743727E40E947437EAEFFFE027
:107200003083303011F40C94891227E40E947437D3
:10721000422EE0E5FFE00FE3040D019300E0008360
:1072200027E40E94743727E40E94743727E40E9401
:10723000743727E40E94743727E40E94743727E4E8
:107240000E94743727E40E94743727E40E94743741
:1072500027E40E94743727E40E94743727E40E94D1
:107260007437022E132E27E40E947437222E332EF9
:10727000000C111C221C331C0FE3040D000E00E057
:10728000101E201E301EECE7FFE0019211922192A9
:1072900030824F903F902F901F900F90FF91EF9171
:1072A0003F912F910F9108950F931F932F933F9329
:1072B000AF93BF93CF93DF93EF93FF930F921F9200
:1072C0002F923F924F935F9311D05F914F913F90D8
:1072D0002F901F900F90FF91EF91DF91CF91BF9171
:1072E000AF913F912F911F910F910895E8E6FFE034
:1072F0000081003069F0013069F0023069F003303C
:1073000069F0043069F0053069F000E00083089509
:107310000C9494390C94B1390C94ED390C94143AC2
:107320000C94983A0C94A93AE0E8FFE00081003010
:1073300009F40895C4E0D0E100E01991011761F467
:107340001991011749F41991011731F418810117A6
:1073500019F400E000830895E8E6FFE001E000830F
:1073600000C00091400F0030E1F023E50E94893613
:1073700026E40E9489362DE20E94893623E50E9488
:10738000893623E40E94893621E30E9489362AE067
:107390000E9489362DE00E94893600E00093400F5C
:1073A000089502E00093680F0091800F0230A1F46D
:1073B000E0916C0FF0916D0F2091640F0E94D03519
:1073C0002091650F0E94D0352091660F0E94D03524
:1073D0002091670F0E94D03500C0E8E5FFE000E093
:1073E000019302E00083EAEFFFE00081E2E5FFE0C5
:1073F0000083E4E6FFE003810F9302810F93018194
:107400000F9300810F93FED1EAEFFFE02081F3DDBF
:107410000F910F910F910F91233009F00895E8E635
:10742000FFE003E0008300C0E0E8FFE000810030FF
:1074300029F4E8E6FFE000E00083089544E6E4E094
:10744000F0E10381003051F40281003039F4018110
:10745000003021F40081041708F4402FE0916C0FF4
:10746000F0916D0FE3DB203021F43E7F341708F4F8
:10747000432FE8E5FFE00181003021F4008104178B
:1074800008F4402F542F403009F40895E0916C0F18
:10749000F0916D0F27E40E94743782DB4A9521F04A
:1074A000232F7EDB4A95B1F7E4E0F0E10081051B74
:1074B000008310E00181010B01830281010B028333
:1074C0000381010B03830081003091F401810030BE
:1074D00079F40281003061F40381003049F4E0E87E
:1074E000FFE000E00083E8E6FFE000E000830895AD
:1074F000E8E5FFE00081051B00830181010B0183AA
:107500000081003019F40181003009F00895E2E5AE
:10751000FFE000810A95008331F4E8E6FFE005E032
:1075200000830C94A93AE8E6FFE004E0008300C081
:107530002FE780DC27FD089526FF0895E8E6FFE0A9
:1075400003E00083E8E5FFE000E0019302E0008350
:107550000895E4E6FFE003810F9302810F93018118
:107560000F9300810F931ED00F901F902F903F908C
:10757000233009F40895243049F4E0E8FFE000E006
:107580000083E8E6FFE000E000830895E4E6FFE022
:107590000082118222823382E8E6FFE001E000836C
:1075A0000C94B139EAE5FFE00081003021F00130B0
:1075B00049F10C945C3B0091400F0030E9F023E46A
:1075C0000E9489362EE40E94893623E40E9489367F
:1075D0002DE20E94893623E50E94893621E30E942C
:1075E00089362AE00E9489362DE00E94893600E023
:1075F0000093400F23E0089501E000935A0F23E029
:107600000C94023BEDB7FEB7339601901190219098
:1076100031900091600F00160091610F10060091EB
:10762000620F20060091630F3006D0F00091FC0F2E
:1076300000160091FD0F10060091FE0F200600912C
:10764000FF0F300609F060F401E0000E00E0101EAC
:10765000201E301E329222921292029225E008954C
:10766000002D0F77000FE8E8FFE0008307E0369475
:107670002794179407940A95D1F7E0E5FFE001916C
:10768000000E0081101E00E0201E301E3F922F923F
:107690001F920F9221E0AFDC0F901F902F903F9030
:1076A000E0E7FFE00192119221923082EAE5FFE0EB
:1076B00002E0008323E00895E0E7FFE001901190ED
:1076C000219030803F922F921F920F9221E093DC05
:1076D0000F910F910F910F91233011F023E0089536
:1076E000E8E8FFE01081103029F027E40E947437A9
:1076F0001A95C9F727E40E947437022E132E27E447
:107700000E947437222E332E0FE030220FEF001626
:1077100061F4101651F4201641F40FE0301629F4EC
:1077200024E000E000935A0F0895EDB7FEB73396BA
:1077300001921192219231920092600F1092610F8A
:107740002092620F3092630F1EEF0091880F101B82
:1077500009F449C001E0000E00E0101E201E301E9A
:1077600027E40E9474372015F1F53115E1F527E47F
:107770000E9474372215B9F53315A9F501E0001AF6
:1077800000E0100A200A300A0092FC0F1092FD0F50
:107790002092FE0F3092FF0F125071F102E0000EA6
:1077A00000E0101E201E301E27E40E9474372015B2
:1077B00019F5311509F527E40E9474372215E1F413
:1077C0003315D1F401E0001A00E0100A200A300A53
:1077D0000092FC0F1092FD0F2092FE0F3092FF0FCF
:1077E0001250E1F609C000E00093FC0F0093FD0F7A
:1077F0000093FE0F0093FF0FEAE5FFE000E0008337
:1078000025E00895EDB7FEB73396019011902190D1
:10781000308002E0001A00E0100A200A300AEAEF85
:10782000FFE00081069529F0000C111C221C331C7E
:10783000F9CFECE7FFE00191000E0191101E0191DC
:10784000201E0081301EEDB7FEB7339601921192D3
:10785000219230820895102E0FEF0DBF00E10EBF70
:10786000012D11240C9489120895E199FECF9FBB3C
:107870008EBBE09A99278DB30895FB01DC0105903A
:107880000D920020E1F70895FB01DC0141505040CA
:1078900030F08D910590801919F40020B9F7881BFC
:1078A000990B0895AA1BBB1B51E107C0AA1FBB1F60
:1078B000A617B70710F0A61BB70B881F991F5A957C
:0C78C000A9F780959095BC01CD010895BA
:00000001FF
